:020000040000FA
:06400000FEEF21F01200AA
:084008009EBA0DEF26F09DA801
:1040100003D09EB8F0EF25F0A4BA52EF25F0A4B873
:0840200035EF25F0110012003C
:06402A0008001041000037
:104030006000000001000000114100008800000045
:10404000160000002741000000040000FE000000F0
:10405000254200009E0000002000000045420000B4
:1040600000020000CE000000134300000003000027
:10407000D2000000E54300006100000001000000E4
:0C408000E64300006200000001000000A8
:024110000000AD
:0F4111000A0D4173736572743A20002C206C699B
:074120006E6520000A0D008E
:09412700013132333435363738EA
:104130002E4353560000003132206269740031363C
:1041400020626974203C2033324D42004578742748
:104150006420444F5320706172746974696F6E00FB
:10416000313620626974203E2033324D42003332B2
:1041700020626974203C2032474200333220626959
:1041800074203C20324742204C42410031362062AC
:104190006974203E2033324D42204C424100457824
:1041A00074276420444F5320706172746974696F7E
:1041B0006E204C424100556E6B6E6F776E207061C1
:1041C00072746974696F6E20005761726E696E67F0
:1041D0003A2077726F6E67206F72206E6F20666F65
:1041E000726D6174004C464E20656E747279006485
:1041F000656C2066696C65000A0D4361726420700D
:10420000726573656E74000A0D4361726420676F96
:104210006E650066696C652E630044415441202040
:054220002020202020F9
:0B4225005357303135382D3030312038
:1042300056657220302E30410000444154416E6E6C
:054240006E6E0000009D
:0B4245000A0D4346444C2056657220D1
:10425000302E30420A0D000A0D493C63723E202D7B
:10426000204964656E7420736563746F72000A0D73
:10427000526E6E6E3C63723E202D2052656164204A
:10428000736563746F72206E6E6E000A0D576E6EEA
:104290006E3C63723E202D205265706561742077FC
:1042A000726974652076616C756573203020746F57
:1042B0002032353520746F20736563746F72206E01
:1042C0006E6E000A0D436F6D7061637420666C61E1
:1042D00073682063617264206E6F742070726573FE
:1042E000656E740031323334350A000A0D46696C4C
:1042F00065206572726F720A0D000A0D46696C6561
:10430000204F4B0D0A004E45575F46494C452E4302
:0343100053560001
:0D431300426F6F74207265636F72642073D7
:104320006563746F723A200042797465207065721B
:1043300020736563746F723A2000536563746F7203
:10434000732070657220636C75737465723A200017
:10435000436F7069657320706572204641543A203E
:10436000004D617820726F6F7420656E747269659C
:10437000733A2000536563746F7273207065722006
:104380004641543A2000526F6F7420736563746F16
:10439000723A20004D6178206469722073656374FD
:1043A0006F72733A20004461746120736563746FA7
:1043B000723A2000464154203120736563746F7255
:1043C0003A2000464154203220736563746F723A7C
:1043D0002000526573657276656420736563746F3F
:0543E00072733A200099
:0243E5000000D6
:0243E6000000D5
:0843E80086801200869012008D
:0C43F000867012008650010B00D01200F5
:0443FC001DEE00F0C2
:104400002DEE00F0F86A189CC1EC22F085EC28F043
:04441000FDD71200C2
:0C4414000C6A0B6A100EE76ED8900F3691
:1044200010360B360C3614500B5C15500C5805E347
:1044300014500B5E15500C5A0F2AE72EF0D71200BD
:104440000C6A0B6A0A6A180EE76ED8900E360F36A1
:1044500010360A360B360C3613500A5C14500B58C3
:1044600015500C5807E313500A5E14500B5A1550A0
:0A4470000C5A0E2AE72EEAD71200BC
:06447A00F26AF168C00EB9
:10448000F06E9E6AA16AA46A9D6AA06AA36A9F6A86
:10449000A26AA56AD08ECD6ACF6ACE6ABA6ABC6AB1
:1044A000BB6AC26A090EC16EC06A070EB46EB56AF5
:1044B000AC6AAB6AAF6A6C6A6B6A6F6A806A2F0E0D
:1044C000926E816AFD0E936E826A930E946E836A79
:1044D0009568E70E846E180E966E100E856E090EA6
:0A44E000976E040E866E986E1200AF
:0644EA00CD6ACF6ACE6A24
:1044F000BA6ABC6ABB6AC26AC16AC06A85909780A0
:10450000809A928A809292828090928080969286FF
:10451000809492840001606B1200D9CFE6FFE1CF56
:10452000D9FF0001605102E0000E25D0CD6A0B0ECC
:10453000BA6EFD0EDBCF00F0FE0EDBCF01F001C046
:1045400000F0016A0050BC6EFF0EE76EFD0EDBCF7F
:1045500000F0FE0EDBCF01F0E7500016016A0050BC
:10456000BB6EC26A090EC16E820EC06EC280CD8063
:104570006069FF0E00D0E552E7CFD9FF120075EF5A
:0245800022F027
:0E4582002A0EF66E400EF76E000EF86E000167
:104590000900F550716F0900F550726F03E1716702
:1045A00001D03DD00900F5506C6F0900F5506D6FDA
:1045B0000900F5506E6F09000900F550E96E090019
:1045C000F550EA6E090009000900F5506F6F090007
:1045D000F550706F09000900F6CF73F0F7CF74F053
:1045E000F8CF75F06CC0F6FF6DC0F7FF6EC0F8FF36
:1045F00000016F5302E1705307E00900F550EE6EC1
:104600006F07F8E27007F9D773C0F6FF74C0F7FFC1
:1046100075C0F8FF00017107000E725BBFD7120072
:10462000D9CFE6FFE1CFD9FFFD0EDBCFE6FFFE0ECF
:10463000DBCFE6FF28EC2AF0E552E5529B0EE66E52
:10464000000EE66E28EC2AF0E552E552E552E7CF7F
:10465000D9FF1200D9CFE6FFE1CFD9FF070EE1263F
:10466000D950FD0FE96EFF0EDA20EA6EEE50ED1024
:104670003AE0880EE66E000EE66E28EC2AF0E5526F
:10468000E552FB0EDBCFE6FFFC0EDBCFE6FF28ECAE
:104690002AF0E552E552930EE66E000EE66E28EC27
:1046A0002AF0E552E552D9CFE6FFDACFE6FFF90E60
:1046B000DBCFE6FFFA0EDBCFE6FFF0EC28F0E106F9
:1046C000E106E106E106D9CFE6FFDACFE6FF28EC06
:1046D0002AF0E552E5529B0EE66E000EE66E28ECDF
:1046E0002AF0E552E552D9CFE1FFE552E7CFD9FFF5
:0246F0001200B6
:0E46F20010C01CF00FC01BF00F501402F4CFCC
:104700000EF0F3CF0DF010501502F4CF10F0F3CFF0
:104710000FF01402F3500E26F4500F22E86A102214
:104720001B501502F3500E26F4500F22E86A102297
:1047300015AE9FEF23F01B500F5E1C50105A1CAE9D
:10474000000C14500F5E1550105A000C0FC01BF0D7
:104750000F501402F4CF0EF0F3CF0DF010501502ED
:10476000F4CF10F0F3CF0FF01402F3500E26F450F4
:104770000F22E86A10221B501502F3500E26F45047
:104780000F22E86A1022000C10C01CF00FC01BF0B2
:104790000EC01AF00E501302F4CF0CF0F3CF0BF052
:1047A0000F501402F4CF0EF0F3CF0DF01302F350BC
:1047B0000C26F4500D22E86A0E221A501402F3500F
:1047C0000C26F4500D22E86A0E2210501302F3500A
:1047D0000D26F4500E22105014020F6AE86A0F22C0
:1047E000F3500E26F4500F221A501502F3500D26E6
:1047F000F4500E22106AE86A0F2210221B50150294
:10480000F3500E26F4500F22E86A10221C501502B5
:0A481000F3500F26F4501022000CA4
:06481A00D9CFE6FFE1CF5B
:10482000D9FFFD0EDB5014E1FE0EDB50030A0DE054
:10483000010A09E0030A05E0010A01E008D09394A7
:1048400006D0939604D0939802D0939A00D013D0B8
:10485000FE0EDB50030A0DE0010A09E0030A05E041
:10486000010A01E008D0938406D0938604D093888F
:1048700002D0938A00D0E552E7CFD9FF1200D9CFFA
:10488000E6FFE1CFD9FFFD0EDB5014E1FE0EDB5059
:10489000030A0DE0010A09E0030A05E0010A01E04C
:1048A00008D0819406D0819604D0819802D0819A54
:1048B00000D013D0FE0EDB50030A0DE0010A09E020
:1048C000030A05E0010A01E008D0818406D0818650
:1048D00004D0818802D0818A00D0E552E7CFD9FF89
:1048E0001200D9CFE6FFE1CFD9FFFE0EDB50030A5D
:1048F0000DE0010A09E0030A05E0010A01E008D021
:10490000817406D0817604D0817802D0817A00D07B
:10491000E552E7CFD9FF1200D9CFE6FFE1CFD9FFAB
:10492000E652DF6AFE0EDB50030A16E0010A0FE0D2
:10493000030A08E0010A01E014D081A402D0010EAC
:10494000DF6E0FD081A602D0010EDF6E0AD081A8E3
:1049500002D0010EDF6E05D081AA02D0010EDF6EFB
:1049600000D0DF5000D0E552E552E7CFD9FF12006A
:10497000D9CFE6FFE1CFD9FF0001625102E0000E7E
:104980001AD00E01686B696B6A6B8B6B8C6B8D6BCD
:104990006C84FE0EDB506F6EA588A58AA38A858A7B
:1049A000858E6C8A6B886B8EFD0EDBCF47FE000117
:1049B0006269FF0E00D0E552E7CFD9FF12006C6AA2
:1049C0006B6AA398A39A829C829E85948596859A09
:1049D000859E0001626B1200D9CFE6FFE1CFD9FFBF
:1049E0000001625114E0200E0E016A5D10E2685170
:1049F000EA6A480FE96E0E0EEA22FE0EDBCFEFFFE9
:104A0000682B1F0E68176A2BA388FF0E02D0000EBA
:104A100000D0E552E7CFD9FF1200D9CFE6FFE1CFB2
:104A2000D9FF000162511BE00E018D51000817E211
:104A30008C51EA6A6B0FE96E0E0EEA22EF50E66EB9
:104A4000FD0EDBCFE9FFFE0EDBCFEAFFE552E750BC
:104A5000EF6E8C2B1F0E8C178D07FF0E02D0000EF1
:104A600000D0E552E7CFD9FF1200E9CFE4FFEACF4B
:104A7000E4FFE6520E016A5100080DE26951EA6A4C
:104A8000480FE96E0E0EEA22EF506D6E692B1F0E75
:104A900069176A0701D0A398E552E5CFEAFFE5CF91
:104AA000E9FF1100E9CFE4FFEACFE4FFE652200E70
:104AB0000E018D5D0DE28B51EA6A6B0FE96E0E0EF1
:104AC000EA226ECFEFFF8B2B1F0E8B178D2B02D0A0
:104AD0006E50E86EE552E5CFEAFFE5CFE9FF110041
:104AE000D9CFE6FFE1CFD9FF0001615102E0000E0E
:104AF0001CD00E01216B226B236B446B456B466B04
:104B0000AC84FE0EDB50AF6E9F889F8A9D8AFD0E9F
:104B1000DBB0858C858A858EAC8AAB88AB8EDBCF8B
:104B200000FE00016169FF0E00D0E552E7CFD9FF1A
:104B30001200AC6AAB6A9D989D9A829C829E859475
:104B40008596859C859A859E0001616B1200D9CF60
:104B5000E6FFE1CFD9FF0001615114E0200E0E0104
:104B6000235D10E22151EA6A010FE96E0E0EEA227E
:104B7000FE0EDBCFEFFF212B1F0E2117232B9D886D
:104B8000FF0E02D0000E00D0E552E7CFD9FF120091
:104B9000D9CFE6FFE1CFD9FF000161511BE00E0143
:104BA0004651000817E24551EA6A240FE96E0E0EDD
:104BB000EA22EF50E66EFD0EDBCFE9FFFE0EDBCF03
:104BC000EAFFE552E750EF6E452B1F0E45174607EB
:104BD000FF0E02D0000E00D0E552E7CFD9FF120041
:104BE000E9CFE4FFEACFE4FFE6520E0123510008CB
:104BF0000DE22251EA6A010FE96E0E0EEA22EF5031
:104C0000AD6E222B1F0E2217230701D09D98E5526F
:104C1000E5CFEAFFE5CFE9FF1100E9CFE4FFEACFF6
:104C2000E4FFE652200E0E01465D0DE24451EA6AB1
:104C3000240FE96E0E0EEA22AECFEFFF442B1F0EBB
:104C40004417462B02D0AE50E86EE552E5CFEAFF9E
:064C5000E5CFE9FF1100B1
:0A4C5600000EE66E020EE66E28EC7A
:104C60002AF0E552E5520001866B876B1200D9CF1E
:104C7000E6FFE1CFD9FF050EE126D9CFE6FFDACF77
:104C8000E6FF0DEC25F0E552E552000901E11AD1ED
:104C9000000EDF9E0D0EDF5C01E004D100018651A5
:104CA000EA6A760FE96E000EEA22EF6A610E765D1F
:104CB00004E376517A0801E3769B760EE66E000EE9
:104CC000E66E73EC2AF0E552E55200017651470A90
:104CD00001E1DED0140A01E1D2D01B0A01E1B6D015
:104CE000770A01E1B3D0680A01E197D0050A76E0BE
:104CF0001B0A67E0020A62E0110A39E0030A18E0C1
:104D0000010A01E0CCD0770EE66E000EE66EB0EC44
:104D100029F0E552E552F3CF00F0F4CF01F000C0E6
:104D2000E6FF01C0E6FF72EC48F0E552E552B7D06D
:104D3000770EE66E000EE66EB0EC29F0E552E55215
:104D4000F3CF00F0F4CF01F000C0E6FF01C0E6FFB2
:104D500070EC3BF0E552E552DF6EDFCFE6FFE66A2E
:104D600048EC2AF0E552E5526AEC2AF098D0770E2A
:104D7000E66E000EE66EB0EC29F0E552E552F3CF98
:104D800000F0F4CF01F000C0E6FF01C0E6FFCFEC79
:104D90003BF0E552E552DE52F3CFDEFFF4CFDDFF0C
:104DA000DD52010EDBCFE6FF020EDBCFE6FF48EC63
:104DB0002AF0E552E5526AEC2AF071D025EC38F081
:104DC0006ED08DEC2DF0000908E07E0EE66E020E2E
:104DD000E66E28EC2AF0E552E55261D0770EE66ED9
:104DE000000EE66EB0EC29F0E552E552F3CF00F08C
:104DF000F4CF01F000C0E6FF01C0E6FFDBEC2CF0D1
:104E0000E552E552000908E07E0EE66E020EE66EFF
:104E100028EC2AF0E552E55242D0770EE66E000EFD
:104E2000E66E88EC29F0E552E552E66EE66A0CEC97
:104E30002EF0E552E552000908E07E0EE66E020E05
:104E4000E66E28EC2AF0E552E55229D0120EE66E05
:104E5000020EE66E28EC2AF0E552E552290EE66EC7
:104E6000020EE66E28EC2AF0E552E552460EE66E9A
:104E7000020EE66E28EC2AF0E552E55210D0770ECD
:104E8000E66E000EE66E58EC31F0E552E55207D0C2
:104E9000A9EC30F005EC31F0F4EC31F000D0000179
:104EA000866B10D00A0EDF5C0DE00F0E0001865DF0
:104EB00009E28651EA6A760FE96E000EEA22DFCF38
:104EC000EFFF862BD9CFE1FFE552E7CFD9FF1200E4
:104ED000D9CFE6FFE1CFD9FFE652D9CFE6FFDACF4F
:104EE000E6FFC8EC25F0E552E552000905E0DFCF0A
:104EF000E6FFA7EC25F0E552E552E552E7CFD9FFF2
:104F00001200D9CFE6FFE1CFD9FFE652D9CFE6FFB5
:104F1000DACFE6FFC8EC25F0E552E552000905E0DE
:104F2000DFCFE6FFECEC24F0E552E552E552E7CFA7
:104F3000D9FF1200D9CFE6FFE1CFD9FF030EE1265A
:104F4000D9CFE6FFDACFE6FFC8EC25F0E552E5520F
:104F5000000901E1D4D0030EDF5C01E0B9D000010B
:104F6000B25101E0B0D0F4EC21F0040100050001E1
:104F7000B26F0E01D451EA6A8E0FE96E0E0EEA226C
:104F80000D0EEF6ED42BD60EE66E0E0EE66E2DECE9
:104F900034F0E552E5521DEC35F0010EDB6ADB50D2
:104FA000EA6AD60FE96E0E0EEA22EF5016E0010E05
:104FB000DB50EA6AD60FE96E0E0EEA22EF50E66E7B
:104FC000010EDB50EA6AB10FE96E0E0EEA22E552DD
:104FD000E750EF6E010EDB2AE2D7010EF36E020EF0
:104FE000F3CFDBFF020EDB50EA6A8E0FE96E0E0E86
:104FF000EA22EF500D0818E0020EDB50EA6A8E0F2D
:10500000E96E0E0EEA22EF50E66E010EDB50EA6A00
:10501000B10FE96E0E0EEA22E552E750EF6E020E76
:10502000DB2A010EDB2ADED7010EDB06DB50EA6A43
:10503000B10FE96E0E0EEA220D0EEF6E010EDB2AA5
:10504000DB50EA6AB10FE96E0E0EEA220A0EEF6E2D
:10505000010EDB2ADBCFE6FFE66AB10EE66E0E0E2E
:10506000E66E000EE66EE66A6AEC45F0F56E060E38
:10507000E15EF5500E01D46BD451EA6AB10FE96ECE
:105080000E0EEA22EF500D080EE0D451EA6AB10F7D
:10509000E96E0E0EEA22EF50E66EECEC24F0E552DB
:1050A0000E01D42BE9D70D0EE66EECEC24F0E552A0
:1050B0000A0EE66EECEC24F0E5520E01D46BD56BD3
:1050C000F6EC21F004D0B2070E01D46BD56B17D0EB
:1050D000020EDF5C05E10E01010ED56FD46B0FD01F
:1050E0000E01D5510CE0210ED45D09E2D451EA6ADB
:1050F0008E0FE96E0E0EEA22DFCFEFFFD42BD9CF51
:10510000E1FFE552E7CFD9FF1200D9CFE6FFE1CFAB
:10511000D9FF020EE1263DEC22F0F28EF29CE66A07
:10512000E66A0DEC24F0E552E552E66A010EE66E01
:105130000DEC24F0E552E552E66A020EE66E0DEC47
:1051400024F0E552E552E66A030EE66E0DEC24F01B
:10515000E552E5527F0EE66E010EE66E8DEC22F012
:10516000E552E552E66A2F0EE66E70EC25F0E55248
:10517000E552E66A170EE66EB8EC24F0E552E55209
:10518000CAEC2CF02BEC26F0ADEC39F00E01D46B10
:105190000E01D56B9E0EE66E000EE66E28EC2AF030
:1051A000E552E552A9EC30F005EC31F0F4EC31F0C9
:1051B00013EC35F01DEC35F00400B1EC39F00009CA
:1051C00002E0B8DE04D00E01D46B0E01D56B37ECD3
:1051D00026F0F2D7D9CFE1FFE552E7CFD9FF120091
:1051E000D9CFE6FFE1CFD9FF050EE126040EDB6A39
:1051F000100EF36E020EF3CFDBFF270EF36E030EDD
:10520000F3CFDBFFD950020FE96EDACFEAFFEE50A1
:10521000ED1071E0FD0EDBCF0FF0FE0EDBCF10F0D6
:10522000020EDBCF14F0030EDBCF15F00AEC22F0F8
:105230000FC0DEFF10C0DDFFD9CFE9FFDACFEAFFF4
:10524000EE50ED100DE1040EDB500AE1D950020FD3
:10525000E96EDACFEAFF010EEE1801E1ED501AE136
:10526000010EF36E040EF3CFDBFFDECF00F0DDCFD7
:1052700001F0300E0026000E0122FB0EDBCFE9FF0D
:10528000FC0EDBCFEAFF00C0EFFFFB0EDB2AFC0EBB
:1052900001E3DB2AFD0EDBCF02F0FE0EDBCF03F0D5
:1052A000020EDBCF0FF0030EDBCF10F0DECF14F0D9
:1052B000DDCF15F0A6EC23F00D50025C006E0E5011
:1052C0000358016EFD0E00C0DBFFFE0E01C0DBFFC8
:1052D000D950020FE96EDACFEAFF0A0E146E156A92
:1052E000EECF0FF0EDCF10F00AEC22F00FC0EEFF82
:1052F00010C0EDFF87D7FB0EDBCFE9FFFC0EDBCF45
:10530000EAFFEF6AD9CFE1FFE552E7CFD9FF1200FC
:10531000D9CFE6FFE1CFD9FFE652DF6AFD0EDBCF42
:10532000E9FFFE0EDBCFEAFFEF5013E00A0EDF02CB
:10533000F3CFDFFFFD0EDBCFE9FFFE0EDBCFEAFF91
:10534000EF50D00FDF26FD0EDB2AFE0E01E3DB2A35
:10535000E5D7DF5000D0E552E552E7CFD9FF120084
:10536000D9CFE6FFE1CFD9FF020EE126DE6ADD6A82
:10537000FD0EDBCFE9FFFE0EDBCFEAFFEF501EE0B4
:10538000D9CFE9FFDACFEAFF0A0EEC02F3CFEDFF47
:10539000EF02F3CFEEFFF450ED26FD0EDBCFE9FF79
:1053A000FE0EDBCFEAFFEF50D00FDE26000EDD222F
:1053B000FD0EDB2AFE0E01E3DB2ADAD7DECF00F09A
:1053C000DDCF01F000C0F3FF01C0F4FF00D0D9CF62
:1053D000E1FFE552E7CFD9FF1200D9CFE6FFE1CFD9
:1053E000D9FFFE0EDBCFE6FFECEC24F0E55200091E
:1053F00001E1F7D7E552E7CFD9FF1200D9CFE6FF99
:10540000E1CFD9FFE652FE0EDB380F0BDF6EDF5027
:10541000090803E2370EDF2602D0300EDF26DFCF89
:10542000E6FFDBDFE552FE0EDB500F0BDF6EDF50D9
:10543000090803E2370EDF2602D0300EDF26DFCF69
:10544000E6FFCBDFE552E552E552E7CFD9FF120088
:10545000D9CFE6FFE1CFD9FFFD0EDBCFE9FFFE0E8E
:10546000DBCFEAFFEF5010E0FD0EDBCFE9FFFE0ED1
:10547000DBCFEAFFEF50E66EB0DFE552FD0EDB2A30
:10548000FE0E01E3DB2AE8D7E552E7CFD9FF120091
:10549000D9CFE6FFE1CFD9FF060EE126D9CFE6FF4F
:1054A000DACFE6FFFD0EDBCFE6FFFE0EDBCFE6FF39
:1054B00097DEE106E106E106E106D9CFE6FFDACFA5
:1054C000E6FFC6DFE552E552D9CFE1FFE552E7CF6F
:1054D000D9FF12000D0EE66E80DFE5520A0EE66E71
:1054E0007CDFE5521200D9CFE6FFE1CFD9FFFD0EF8
:1054F000DBCFE6FFFE0EDBCFE6FFAADFE552E5528B
:10550000E9DFE552E7CFD9FF1200D9CFE6FFE1CFBF
:10551000D9FF020EE126FD0EDB2AFE0E01E3DB2A97
:10552000FD0EDBCFE9FFFE0EDBCFEAFFEF50DE6EB4
:10553000DD6AD9CFE9FFDACFEAFFF0CFEFFFF06AFB
:10554000FD0EDB06FE0E01E2DB06FD0EDBCFE9FF02
:10555000FE0EDBCFEAFFEF50DE26000EDD22DECFAF
:1055600000F0DDCF01F000C0F3FF01C0F4FF00D078
:10557000D9CFE1FFE552E7CFD9FF1200D9CFE6FF3F
:10558000E1CFD9FF070EE126060EDB6A100EF36E9F
:10559000030EF3CFDBFF270EF36E040EF3CFDBFF1A
:1055A000050EDB6A030EDBCF00F0040EDBCF01F04B
:1055B000050EDBCF02F000500110021001E1A8D06F
:1055C000FC0EDBCF00F0FD0EDBCF01F0FE0EDBCFDB
:1055D00002F000C00EF001C00FF002C010F0030E88
:1055E000DBCF13F0040EDBCF14F0050EDBCF15F08C
:1055F00020EC22F00EC0DFFF010E0FC0DBFF020E19
:1056000010C0DBFFDFCF00F0010EDBCF01F0020E98
:10561000DBCF02F00050011002100FE1060EDB504C
:105620000CE1D950030FE96EDACFEAFF010EEE1854
:1056300003E1EE5001E1EE501FE1010EF36E060EA4
:10564000F3CFDBFFDFCF00F0010EDBCF01F0020E66
:10565000DBCF02F0300E0026000E01220222FA0EED
:10566000DBCFE9FFFB0EDBCFEAFF00C0EFFFFA0E56
:10567000DB2AFB0E01E3DB2AFC0EDBCF03F0FD0E81
:10568000DBCF04F0FE0EDBCF05F0DFCF06F0010E1E
:10569000DBCF07F0020EDBCF08F006C00EF007C02C
:1056A0000FF008C010F0030EDBCF13F0040EDBCFB9
:1056B00014F0050EDBCF15F0C4EC23F00B50035CA7
:1056C000006E0C500458016E0D500558026EFC0E11
:1056D00000C0DBFFFD0E01C0DBFFFE0E02C0DBFFE2
:1056E000D950030FE96EDACFEAFF0A0E136E146A7F
:1056F000156AEECF0EF0EECF0FF0EFCF10F020ECEA
:1057000022F010C0EDFF0FC0EDFF0EC0EFFF4AD733
:10571000FA0EDBCFE9FFFB0EDBCFEAFFEF6AD9CF52
:0A572000E1FFE552E7CFD9FF1200C8
:06572A00D9CFE6FFE1CF3C
:10573000D9FFE65284A8FED71F0E8416FE0EDB505A
:10574000E00B84128490000000008350DF6E8480A0
:10575000DF5000D0E552E552E7CFD9FF1200D9CF94
:10576000E6FFE1CFD9FF84A8FED7FD0EDB50836EA4
:105770001F0E8416FE0EDB50E00B84128492000094
:1057800000008482E552E7CFD9FF1200D9CFE6FFAF
:10579000E1CFD9FFFE0EDB380F0BF36EFE0EF3CF19
:1057A000DBFFDB5009080BE2370E006EFE0EDBCF8D
:1057B000E7FF0050E726FE0EE7CFDBFF0AD0300EF2
:1057C000006EFE0EDBCFE7FF0050E726FE0EE7CFB0
:1057D000DBFFFE0EDBCFE6FFECEC24F0E552000928
:1057E00001E1F7D7E552E7CFD9FF1200D9CFE6FFA5
:1057F000E1CFD9FFFE0EDB98DB9ADB9CDB9EFE0E31
:10580000DB5009080BE2370E006EFE0EDBCFE7FF20
:105810000050E726FE0EE7CFDBFF0AD0300E006E09
:10582000FE0EDBCFE7FF0050E726FE0EE7CFDBFFE3
:10583000FE0EDBCFE6FFECEC24F0E552000901E1BF
:10584000F7D7E552E7CFD9FF1200D9CFE6FFE1CF76
:10585000D9FF030EE126FD0EDBCF0FF0FE0EDBCFEE
:1058600010F0DE520FC0DEFF10C0DDFFDD52DF6A38
:10587000100EDF5C3AE2FD0EDBCFE9FFFE0EDBCF60
:10588000EAFFEF50E66E82DFE552FD0EDBCFE9FF67
:10589000FE0EDBCFEAFFEF50E66EA8DFE552FD0E0D
:1058A000DB2AFE0E01E3DB2AFD0EDBCFE9FFFE0E55
:1058B000DBCFEAFFEF50E66E69DFE552FD0EDBCF8E
:1058C000E9FFFE0EDBCFEAFFEF50E66E8FDFE55219
:1058D000FD0EDB2AFE0E01E3DB2A200EE66EEDEC68
:1058E00029F0E552020EDF26C3D7010EDBCF0FF001
:1058F000020EDBCF10F0FD0E0FC0DBFFFE0E10C05E
:10590000DBFFDF6A100EDF5C2CE2FD0EDBCFE9FF70
:10591000FE0EDBCFEAFFEFCF00F0200E005C15E3B8
:10592000FD0EDBCFE9FFFE0EDBCFEAFFEF507E0876
:105930000CE3FD0EDBCFE9FFFE0EDBCFEAFFEF50FD
:10594000E66EEDEC29F0E55205D02E0EE66EEDEC9C
:1059500029F0E552FD0EDB2AFE0E01E3DB2ADF2AE9
:10596000D1D70D0EE66EEDEC29F0E5520A0EE66E8B
:10597000EDEC29F0E552D9CFE1FFE552E7CFD9FFB1
:10598000120084A603D08588000E03D08598FF0EF0
:1059900000D012008588979884949694848096907D
:1059A0008482969296869688836A956A1F0E8416DC
:1059B000961685981200D9CFE6FFE1CFD9FF140ED5
:1059C000E126130EDB6ADDDF000901E198D0956A5C
:1059D000E00EE66EC00EE66EC2DEE552E552E66A05
:1059E000A00EE66EBCDEE552E552FD0EDBCF00F008
:1059F000FE0EDBCF01F001C000F0016A0050E66E40
:105A0000800EE66EACDEE552E552FF0EE76EFD0E4F
:105A1000DBCF00F0FE0EDBCF01F0E7500016016A8D
:105A20000050E66E600EE66E9ADEE552E552010E1B
:105A3000E66E400EE66E93DEE552E552200EE66E0F
:105A4000E00EE66E8CDEE552E55295681F0E841678
:105A5000100EDB6A110EDB6A120EDB6A110EDBCF51
:105A600000F0120EDBCF01F0000E005C020E0158B8
:105A700044E2E66A5ADEE552E66ED9CF00F0DACFAC
:105A800001F0100EDB500F01EA6B0024E96F0150AA
:105A9000EA23E552E750EF6E100EDB2A110EDB2AE7
:105AA000120E01E3DB2AE66A40DEE552E66ED9CF4C
:105AB00000F0DACF01F0100EDB500F01EA6B00248A
:105AC000E96F0150EA23E552E750EF6E100EDB2A32
:105AD000F36EDBCFF4FFF350F45C09E3D9CFE6FFBC
:105AE000DACFE6FFB2DEE552E552100EDB6A110EA8
:105AF000DB2A120E01E3DB2AB1D7956A05D0010E2D
:105B0000F36E130EF3CFDBFF130EDB5000D0D9CFB3
:105B1000E1FFE552E7CFD9FF1200D9CFE6FFE1CF91
:105B2000D9FF160EE126150EDB6A2BDF000966E0B1
:105B3000956AEC0EE66EE00EE66E11DEE552E55279
:105B400095681F0E8416040EDB6ADE6ADD6ADECFFE
:105B500000F0DDCF01F0000E005C020E01584CE2B7
:105B6000E66AE3DDE552E76E030EE7CFDBFFDF2AEF
:105B7000010E01E3DB2AE66AD8DDE552E76E020E8C
:105B8000E7CFDBFFD950050F006EDACF01F0040E2E
:105B9000DB500F01EA6B0024E96F0150EA23020E8B
:105BA000DBCFEFFF040EDB2AD950050F006EDACFF2
:105BB00001F0040EDB50EA6B0024E96F0150EA2388
:105BC000030EDBCFEFFF040EDB2A100EF36E040E84
:105BD000DBCFF4FFF350F45C0AE3D950050FE66E17
:105BE000DACFE6FF32DEE552E552040EDB6ADF2A49
:105BF000010E01E3DB2AABD7956A05D0010EF36EE7
:105C0000150EF3CFDBFF150EDB5000D0D9CFE1FF2F
:105C1000E552E7CFD9FF1200D9CFE6FFE1CFD9FF98
:105C2000040EE126030EDB6AACDE00095CE0956A37
:105C3000E00EE66EC00EE66E92DDE552E552E66AD3
:105C4000A00EE66E8CDDE552E552FD0EDBCF00F0D6
:105C5000FE0EDBCF01F001C000F0016A0050E66EDD
:105C6000800EE66E7CDDE552E552FF0EE76EFD0E1E
:105C7000DBCF00F0FE0EDBCF01F0E7500016016A2B
:105C80000050E66E600EE66E6ADDE552E552010EEA
:105C9000E66E400EE66E63DDE552E552300EE66ECE
:105CA000E00EE66E5CDDE552E5521F0E8416020E34
:105CB000DB6ADE6ADD6ADECF00F0DDCF01F0000EC8
:105CC000005C020E01580EE2020EDBCFE6FFE66A30
:105CD00046DDE552E552020EDB2ADF2A010E01E322
:105CE000DB2AE9D705D0010EF36E030EF3CFDBFFFD
:105CF000030EDB5000D0D9CFE1FFE552E7CFD9FF4B
:105D00001200D9CFE6FFE1CFD9FF030EE126020E44
:105D1000DB6A820E006E590E016E005001106AE0BF
:105D2000956AE00EE66EC00EE66E19DDE552E552AC
:105D3000E66AA00EE66E13DDE552E552FD0EDBCFFE
:105D400000F0FE0EDBCF01F001C000F0016A005050
:105D5000E66E800EE66E03DDE552E552FF0EE76E5D
:105D6000FD0EDBCF00F0FE0EDBCF01F0E75000169A
:105D7000016A0050E66E600EE66EF1DCE552E55217
:105D8000010EE66E400EE66EEADCE552E552200EAC
:105D9000E66EE00EE66EE3DCE552E55295681F0E16
:105DA0008416DE6ADD6ADECF00F0DDCF01F0FB0E87
:105DB000DBCF02F0FC0EDBCF03F00250005C03509F
:105DC000015817E2E66AB1DCE552E66EF90EDBCF68
:105DD000E9FFFA0EDBCFEAFFE552E750EF6EF90E6E
:105DE000DB2AFA0E01E3DB2ADF2A010E01E3DB2ABC
:105DF000DAD705D0010EF36E020EF3CFDBFF020EF1
:105E0000DB5000D0D9CFE1FFE552E7CFD9FF120038
:105E1000D9CFE6FFE1CFD9FF030EE126020EDB6A00
:105E2000820E006E590E016E0050011029E0DE6AEC
:105E3000DD6ADECF00F0DDCF01F0FD0EDBCF02F03A
:105E4000FE0EDBCF03F00250005C0350015817E256
:105E5000E66A6BDCE552E66EFB0EDBCFE9FFFC0E7B
:105E6000DBCFEAFFE552E750EF6EFB0EDB2AFC0EBC
:105E700001E3DB2ADF2A010E01E3DB2ADAD705D0B2
:105E8000010EF36E020EF3CFDBFF020EDB5000D0EB
:105E9000D9CFE1FFE552E7CFD9FF1200D9CFE6FF16
:105EA000E1CFD9FF030EE126020EDB6A820E006EFF
:105EB000590E016E0050011069E0956AE00EE66E21
:105EC000C00EE66E4CDCE552E552E66AA00EE66EC8
:105ED00046DCE552E552FD0EDBCF00F0FE0EDBCFD7
:105EE00001F001C000F0016A0050E66E800EE66E1F
:105EF00036DCE552E552FF0EE76EFD0EDBCF00F01B
:105F0000FE0EDBCF01F0E7500016016A0050E66E8E
:105F1000600EE66E24DCE552E552010EE66E400EA0
:105F2000E66E1DDCE552E552300EE66EE00EE66EE2
:105F300016DCE552E5521F0E8416DE6ADD6ADECFFE
:105F400000F0DDCF01F0FB0EDBCF02F0FC0EDBCF6B
:105F500003F00250005C0350015817E2F90EDBCF4A
:105F6000E9FFFA0EDBCFEAFFEF50E66EE66AAFEC30
:105F70002BF0E552E552F90EDB2AFA0E01E3DB2A9B
:105F8000DF2A010E01E3DB2ADAD705D0010EF36E1A
:105F9000020EF3CFDBFF020EDB5000D0D9CFE1FFC2
:105FA000E552E7CFD9FF1200D9CFE6FFE1CFD9FF05
:105FB000030EE126020EDB6A820E006E590E016EA0
:105FC0000050011029E0DE6ADD6ADECF00F0DDCF8F
:105FD00001F0FD0EDBCF02F0FE0EDBCF03F002502E
:105FE000005C0350015817E2FB0EDBCFE9FFFC0E0B
:105FF000DBCFEAFFEF50E66EE66AAFEC2BF0E5523E
:10600000E552FB0EDB2AFC0E01E3DB2ADF2A010E40
:1060100001E3DB2ADAD705D0010EF36E020EF3CFCF
:10602000DBFF020EDB5000D0D9CFE1FFE552E7CF16
:04603000D9FF120082
:0C6034000000000000000000120082923A
:10604000F9DF829012008292F5DF8280F3DF828294
:106050001200D9CFE6FFE1CFD9FF020EE126010EF3
:10606000DF6EDB6A080EF36E010EDBCFF4FFF35038
:10607000F45C20E2010EDBCFE6FF070EE552D8808C
:10608000E754006EFE0EDB5000C0E7FFE75204E06D
:10609000E8427F0BE706FCE1010BF36EF346FD0ED1
:1060A0008214F310826EC6DF8280C4DF8290010EFC
:1060B000DB2AD8D79482BEDF8280BCDF8250020BFD
:1060C00001E0010EDF6E82909492DF5002E1FF0E3C
:1060D00002D0000E00D0D9CFE1FFE552E7CFD9FFC3
:1060E0001200D9CFE6FFE1CFD9FF020EE12694825C
:1060F0008290A0DF010EDB6A080EF36E010EDBCF8B
:10610000F4FFF350F45C0EE2DF9EDF46828092DF04
:106110008250020B01E0010EDF2682908BDF010E20
:10612000DB2AEAD79492FE0EDB50010B010BF36ED3
:10613000F346FD0E8214F310826E7CDF82807ADFDC
:106140008290DF5000D0D9CFE1FFE552E7CFD9FFF1
:106150001200D9CFE6FFE1CFD9FF160EE126D00E0F
:10616000DF6E020EDB6A030EDB6AD950040FE96EA4
:10617000DACFEAFF0A0EEE6E0D0EEE6E490EEE6EEF
:106180006E0EEE6E690EEE6E740EEE6E690EEE6EB3
:10619000610EEE6E6C0EEE6E690EEE6E730EEE6EAE
:1061A000650EEE6E640EEE6E200EEE6E520EEE6E0C
:1061B000540EEE6E430EEE6EEE6A949094928290C0
:1061C0008282828037DF3BDFDFCFE6FF42DFE552AE
:1061D000E76E020EE7CFDBFFDB5009E0030EDBCFFB
:1061E000E6FF37DFE552E76E020EE7CFDBFF2BDF7E
:1061F000020EDB5002E0FF0E02D0000E00D0D9CF1D
:10620000E1FFE552E7CFD9FF1200D9CFE6FFE1CF9A
:10621000D9FF030EE126D10EDF6E010EDB6AF36EAD
:10622000020EF3CFDBFF0BDFDFCFE6FF12DFE5521D
:10623000E76E020EE7CFDBFFDB5033E0010EDBCF72
:10624000E6FF4FDFE5520001636F010EDBCFE6FF93
:1062500048DFE5520001646F010EDBCFE6FF41DF4E
:10626000E5520001656F010EDBCFE6FF3ADFE55234
:106270000001666F010EDBCFE6FF33DFE552000160
:10628000676F010EDBCFE6FF2CDFE5520001686F80
:10629000DE52010EDD6EDBCFE6FF23DFE5520001AB
:1062A000696FD1DED9CFE1FFE552E7CFD9FF120008
:1062B000D9CFE6FFE1CFD9FF0B0EE126D00EDF6E7E
:1062C000DE52010EDD6E030EDB6A020EDB6AFD0E8E
:1062D000DBCFE9FFFE0EDBCFEAFFEF504CE0FD0E17
:1062E000DBCFE9FFFE0EDBCFEAFFEF50D00FE66E0B
:1062F000D950040F006EDACF01F0020EDB500F010F
:10630000EA6B0024E96F0150EA23E552E750EF6E93
:10631000D950040F006EDACF01F0020EDB50EA6BA9
:106320000024E96F0150EA23EF38F00BEF6EFD0E09
:10633000DB2AFE0E01E3DB2AFD0EDBCFE9FFFE0EBA
:10634000DBCFEAFFEF50D00F026ED950040F006E82
:10635000DACF01F0020EDB50EA6B0024E96F015046
:10636000EA230250EF26FD0EDB2AFE0E01E3DB2AB4
:10637000020EDB2AACD763DEDFCFE6FF6ADEE55232
:10638000E76E010EE7CFDBFFDB5009E0030EDBCF4A
:10639000E6FF5FDEE552E76E010EE7CFDBFF020EA0
:1063A000DB6A070EF36E020EDBCFF4FFF350F45CF2
:1063B00014E2D950040F006EDACF01F0020EDB5068
:1063C0000F01EA6B0024E96F0150EA23EF50E66EFB
:1063D00040DEE552020EDB2AE4D735DED9CFE1FFFD
:1063E000E552E7CFD9FF1200D9CFE6FFE1CFD9FFC1
:1063F0002D0EE126D9CFE9FFDACFEAFF0A0EEE6EC5
:106400000D0EEE6E430EEE6E6F0EEE6E6E0EEE6EB7
:10641000730EEE6E740EEE6E720EEE6E750EEE6E06
:10642000630EEE6E740EEE6E690EEE6E6E0EEE6E16
:10643000670EEE6E200EEE6E440EEE6E610EEE6E88
:10644000740EEE6E650EEE6E200EEE6E610EEE6E4A
:106450006E0EEE6E640EEE6E200EEE6E540EEE6E4E
:10646000690EEE6E6D0EEE6E650EEE6E0A0EEE6E3F
:106470000D0EEE6EEE6A000163390F0B0A0DF3503C
:10648000E66ED9501F0FE96EDACFEAFFE552E7500A
:10649000EE6EED6A0F0E6315006E016AD9501F0F84
:1064A000E96EDACFEAFF0050EE260150ED226439A2
:1064B0000F0B0A0DF350E66ED950210FE96EDACFBB
:1064C000EAFFE552E750EE6EED6A0F0E6415006EBE
:1064D000016AD950210FE96EDACFEAFF0050EE26AB
:1064E0000150ED2265390F0B030B0A0DF350E66ED8
:1064F000D950230FE96EDACFEAFFE552E750EE6E8E
:10650000ED6A0F0E6515006E016AD950230FE96E12
:10651000DACFEAFF0050EE260150ED2267390F0B6B
:106520000A0DF350E66ED950270FE96EDACFEAFF75
:10653000E552E750EE6EED6A0F0E6715006E016AC8
:10654000D950270FE96EDACFEAFF0050EE2601504E
:10655000ED2268390F0B010B0A0DF350E66ED9508E
:10656000290FE96EDACFEAFFE552E750EE6EED6AE9
:106570000F0E6815006E016AD950290FE96EDACF47
:10658000EAFF0050EE260150ED2269390F0B0A0D8B
:10659000F350E66ED9502B0FE96EDACFEAFFE552E1
:1065A000E750EE6EED6A0F0E6915006E016AD95064
:1065B0002B0FE96EDACFEAFF0050EE260150ED22F4
:1065C000D9502B0FE96EDACFEAFFD00EEE26070E78
:1065D000ED22D9CFE6FFDACFE6FF28EC2AF0E5522C
:1065E000E552230EDBCFE6FF240EDBCFE6FF48ECBF
:1065F0002AF0E552E5523A0EE66EEDEC29F0E5524E
:10660000D950210FE96EDACFEAFF090ED880EE5497
:10661000000EED5405E3300EE66EEDEC29F0E55288
:10662000210EDBCFE6FF220EDBCFE6FF48EC2AF09F
:10663000E552E5523A0EE66EEDEC29F0E552D950FE
:106640001F0FE96EDACFEAFF090ED880EE54000E74
:10665000ED5405E3300EE66EEDEC29F0E5521F0E29
:10666000DBCFE6FF200EDBCFE6FF48EC2AF0E55259
:10667000E552200EE66EEDEC29F0E552270EDBCF59
:10668000E6FF280EDBCFE6FF48EC2AF0E552E552A4
:106690002D0EE66EEDEC29F0E552290EDBCFE6FF7C
:1066A0002A0EDBCFE6FF48EC2AF0E552E5522D0E2C
:1066B000E66EEDEC29F0E5522B0EDBCFE6FF2C0E5B
:1066C000DBCFE6FF48EC2AF0E552E552D9CFE1FFF7
:1066D000E552E7CFD9FF1200D9CFE6FFE1CFD9FFCE
:1066E00038DD93DDFD0EDBCFE9FFFE0EDBCFEAFFE9
:1066F000320EEF6EFD0EDB2AFE0E01E3DB2AFD0EED
:10670000DBCFE9FFFE0EDBCFEAFF300EEF6EFD0EB2
:10671000DB2AFE0E01E3DB2A000169390F0B300F83
:10672000E66EFD0EDBCFE9FFFE0EDBCFEAFFE552A2
:10673000E750EF6EFD0EDB2AFE0E01E3DB2A0F0EA3
:106740006915300FE66EFD0EDBCFE9FFFE0EDBCFE5
:10675000EAFFE552E750EF6EFD0EDB2AFE0E01E385
:10676000DB2A68390F0B010B300FE66EFD0EDBCF15
:10677000E9FFFE0EDBCFEAFFE552E750EF6EFD0EBC
:10678000DB2AFE0E01E3DB2A0F0E6815300FE66EE2
:10679000FD0EDBCFE9FFFE0EDBCFEAFFE552E7504F
:1067A000EF6EFD0EDB2AFE0E01E3DB2A67390F0BCD
:1067B000300FE66EFD0EDBCFE9FFFE0EDBCFEAFF0A
:1067C000E552E750EF6EFD0EDB2AFE0E01E3DB2AF9
:1067D0000F0E6715300FE66EFD0EDBCFE9FFFE0EE4
:1067E000DBCFEAFFE552E750EF6EFD0EDB2AFE0E2F
:1067F00001E3DB2AFD0EDBCFE9FFFE0EDBCFEAFF74
:106800002E0EEF6EFD0EDB2AFE0E01E3DB2AFD0EDF
:10681000DBCFE9FFFE0EDBCFEAFF430EEF6EFD0E8E
:10682000DB2AFE0E01E3DB2AFD0EDBCFE9FFFE0EC5
:10683000DBCFEAFF530EEF6EFD0EDB2AFE0E01E307
:10684000DB2AFD0EDBCFE9FFFE0EDBCFEAFF560EA3
:10685000EF6EE552E7CFD9FF1200D9CFE6FFE1CFC7
:10686000D9FF060EE12675DCD0DC000165390F0B7F
:10687000030B0A0DF3CF00F0016A026A00C0DFFFCC
:10688000010E01C0DBFF020E02C0DBFFD9CFE9FF22
:10689000DACFEAFF100E136E0E0E146E156AEECFED
:1068A0000EF0EECF0FF0EFCF10F0C4EC23F00DC0E0
:1068B000EDFF0CC0EDFF0BC0EFFF0F0E00016515E3
:1068C000006E016A026A030E00C0DBFF040E01C005
:1068D000DBFF050E02C0DBFFD950030FE96EDACFF4
:1068E000EAFF100E136E0E0E146E156AEECF0EF048
:1068F000EECF0FF0EFCF10F0C4EC23F00DC0EDFFA2
:106900000CC0EDFF0BC0EFFFD9CFE9FFDACFEAFFF4
:10691000030EDB50EE26040EDB50EE22050EDB509C
:10692000EE22000164390F0B0A0DF3CF00F0016A6B
:10693000026A030E00C0DBFF040E01C0DBFF050E80
:1069400002C0DBFF0F0E6415006E016A026AD950A7
:10695000030FE96EDACFEAFF0050EE260150EE2277
:106960000250EE22D950030FE96EDACFEAFF3C0E57
:10697000136E146A156AEECF0EF0EECF0FF0EFCF64
:1069800010F0C4EC23F00DC0EDFF0CC0EDFF0BC008
:10699000EFFFD9CFE9FFDACFEAFF030EDB50EE2697
:1069A000040EDB50EE22050EDB50EE2200016339AF
:1069B0000F0B0A0DF3CF00F0016A026AD9CFE9FF8D
:1069C000DACFEAFF0050EE260150EE220250EE220E
:1069D0000F0E6315006E016A026AD9CFE9FFDACFA4
:1069E000EAFF0050EE260150EE220250EE22FD0E8C
:1069F000DBCFE6FFFE0EDBCFE6FFD9CFE9FFDACF34
:106A0000EAFFEECFE6FFEECFE6FFEFCFE6FFBEEC0C
:106A10002AF0F56E050EE15EF550D9CFE1FFE552A3
:106A2000E7CFD9FF1200000167390F0B0A0DF3CF32
:106A30006AF00F0E67156A271200D9CFE6FFE1CF83
:106A4000D9FFE652000167390F0B0A0DF350DF6ED4
:106A50000F0E6715DF266A51DF5C02E10101006B52
:106A600000016A51DF5C0AE06B5108E00101010E90
:106A7000006FDFCF6AF000016B6B07D06A51DF5CFB
:106A800004E06B5102E1010E6B6FE552E552E7CF76
:046A9000D9FF120018
:0C6A9400D9CFE6FFE1CFD9FFE652DF6A60
:106AA000100EDF5C1EE2DF50EA6A280FE96E010E6D
:106AB000EA22EF50E66EFEEC29F0E552DF2ADF50C5
:106AC000EA6A280FE96E010EEA22EF50E66EFEEC4C
:106AD00029F0E552DF2A200EE66EEDEC29F0E552B2
:106AE000DFD70D0EE66EEDEC29F0E5520A0EE66EEC
:106AF000EDEC29F0E552E552E552E7CFD9FF12005F
:106B0000D9CFE6FFE1CFD9FFE65201014A6B280E4B
:106B1000E66E010EE66E100EE66EE66A000EE66E9A
:106B2000E66A81EC2EF0F56E060EE15EF550010E80
:106B3000DF6E1C0EDF5C0FE2280EE66E010EE66EC5
:106B4000100EE66EE66A08EC2FF0E106E106E106BB
:106B5000E106DF2AEED7800E0101365D20E1010E4D
:106B60004A6F280EE66E010EE66E100EE66EE66ABD
:106B700008EC2FF0E106E106E106E106040E010152
:106B80002A5D06E0060E2A5D03E00E0E2A5D05E191
:106B90002EC138F12FC139F101D04A6B04D0010E5A
:106BA0004A6F386B396B4A516EE0280EE66E010E63
:106BB000E66E100EE66EE66A38C1E6FF39C1E6FF02
:106BC00081EC2EF0F56E060EE15EF5502B0EE66EB2
:106BD000010EE66E73EC2AF0E552E55233C145F141
:106BE00034C146F135C147F136C148F137C149F1E9
:106BF000280EE66E010EE66E100EE66EE66A08ECF2
:106C00002FF0E106E106E106E10628C13AF129C1CB
:106C10003BF12AC13CF12EC13FF12FC140F13FC1F0
:106C200002F040C103F0D890023603360250010151
:106C30003825006E03503921016E00504825416F00
:106C400001504921426F3BC100F03CC101F0050EEB
:106C5000D89000360136E806FBE100C00FF001C015
:106C600010F045C114F046C115F00AEC22F00FC037
:106C70003DF110C03EF1010141513D25436F4251AC
:106C80003E21446F08D0A20EE66E040EE66E73EC51
:106C90002AF0E552E552E552E552E7CFD9FF12005E
:106CA000D9CFE6FFE1CFD9FF0A0EE126FD0EDBCFFB
:106CB0000FF0FE0EDBCF10F0050E0FC0DBFF060E4F
:106CC00010C0DBFFFD0EDBCFE6FFFE0EDBCFE6FFE5
:106CD00048EC2AF0E552E5522D0EE66EEDEC29F077
:106CE000E552040E01015D6F5E6BDF6AEA6BDF3413
:106CF000FE0BEA36E96E5D0EE926010EEA22050E6C
:106D0000DBCFEEFF060EDBCFEDFFDF2A3851482543
:106D1000006E39514921016E010E00C0DBFF020EE9
:106D200001C0DBFF280EE66E010EE66E100EE66E69
:106D3000E66A010EDBCFE6FF020EDBCFE6FF81EC59
:106D40002EF0F56E060EE15EF550080EDB6A090EB8
:106D5000DB6A070EDB6A070EDB5001E098D0180EE5
:106D6000DF5C01E394D0FD0EDBCF00F0FE0EDBCF45
:106D700001F0080E005C000E015821E3D950FD0F10
:106D8000E96EFF0EDA20EA6E080EEE5E000EED5A96
:106D9000280EE66E010EE66E100EE66EE66A08EC50
:106DA0002FF0E106E106E106E106D950080FE96E91
:106DB000DACFEAFF080EEE26000EED22D4D7FD0E44
:106DC000DBCFE9FFFE0EDBCFEAFFD890E936EA36EB
:106DD000280EE926010EEA22050EEECFDBFF060E95
:106DE000EDCFDBFFD950050FE96EDACFEAFFEF0EEA
:106DF000D880EE54000EED5416E2010EF36E070E2D
:106E0000F3CFDBFF5D0EE66EEDEC29F0E552EA6BA9
:106E1000DF34FE0BEA36E96E5D0EE926010EEA224A
:106E2000EE6AED6A1FD0050EDBCFE6FF060EDBCF64
:106E3000E6FF48EC2AF0E552E5522D0EE66EEDEC49
:106E400029F0E552EA6BDF34FE0BEA36E96E5D0E9F
:106E5000E926010EEA22050EDBCFEEFF060EDBCFA0
:106E6000EDFFDF2A050EDBCF02F0060EDBCF03F0CD
:106E7000080EDB50025C006E090EDB500358016EF9
:106E8000FD0E00C0DBFFFE0E01C0DBFF64D7D9CFD3
:106E9000E1FFE552E7CFD9FF1200D9CFE6FFE1CFFE
:106EA000D9FF0C0EE126FD0EDBCF0FF0FE0EDBCF7F
:106EB00010F0020E0FC0DBFF030E10C0DBFF01015C
:106EC00038514825006E39514921016E00C0DEFF5E
:106ED00001C0DDFFFD0EDBCF00F0FE0EDBCF01F0C9
:106EE000000E005C010E015814E3D950FD0FE96E4D
:106EF000FF0EDA20EA6EEE52ED06D950040FE96E6D
:106F0000DACFEAFFEE52ED2ADF2A010E01E3DB2A97
:106F1000E1D7280EE66E010EE66E100EE66EE66A0A
:106F2000DECFE6FFDDCFE6FF81EC2EF0F56E060E3C
:106F3000E15EF550040EDB6A050EDB6AFD0EDBCF69
:106F400000F0FE0EDBCF01F0080E005C000E0158D1
:106F500021E3D950FD0FE96EFF0EDA20EA6E080E2C
:106F6000EE5E000EED5A280EE66E010EE66E100E75
:106F7000E66EE66A08EC2FF0E106E106E106E106BE
:106F8000D950040FE96EDACFEAFF080EEE26000EA4
:106F9000ED22D4D7FD0EDBCFE9FFFE0EDBCFEAFFFB
:106FA000D890E936EA36280EE926010EEA22020ECA
:106FB000EECFDBFF030EEDCFDBFFD950020FE96E02
:106FC000DACFEAFFEECF00F0EFCF01F0026A036AFA
:106FD000080E00C0DBFF090E01C0DBFF0A0E02C075
:106FE000DBFF0B0E03C0DBFFD950080FE96EDACFD1
:106FF000EAFFEF0ED880EE54FF0EEE54000EEE5472
:10700000000EEE5405E2060EDB6A070EDB6A0CD0BA
:10701000020EDBCF0FF0030EDBCF10F0060E0FC019
:10702000DBFF070E10C0DBFF060EDBCF00F0070E04
:10703000DBCF01F000C0F3FF01C0F4FF00D0D9CFD7
:10704000E1FFE552E7CFD9FF1200D9CFE6FFE1CF4C
:10705000D9FF080EE126150EE66E030EE66E28EC4B
:107060002AF0E552E552D9CFE6FFDACFE6FF45C177
:10707000E6FF46C1E6FFF0EC28F0E106E106E10696
:10708000E106D9CFE6FFDACFE6FF73EC2AF0E5524E
:10709000E552270EE66E030EE66E28EC2AF0E55266
:1070A000E552D9CFE6FFDACFE6FF01014751E66EA0
:1070B000E66AF0EC28F0E106E106E106E106D9CF48
:1070C000E6FFDACFE6FF73EC2AF0E552E552BF0E99
:1070D000E66E030EE66E28EC2AF0E552E552D9CFB3
:1070E000E6FFDACFE6FF48C1E6FF49C1E6FFF0EC74
:1070F00028F0E106E106E106E106D9CFE6FFDACFA6
:10710000E6FF73EC2AF0E552E5523D0EE66E030E03
:10711000E66E28EC2AF0E552E552D9CFE6FFDACF49
:10712000E6FF01013A51E66EE66AF0EC28F0E1066E
:10713000E106E106E106D9CFE6FFDACFE6FF73EC20
:107140002AF0E552E5524E0EE66E030EE66E28EC8E
:107150002AF0E552E552D9CFE6FFDACFE6FF3BC190
:10716000E6FF3CC1E6FFF0EC28F0E106E106E106AF
:10717000E106D9CFE6FFDACFE6FF73EC2AF0E5525D
:10718000E552610EE66E030EE66E28EC2AF0E5523B
:10719000E552D9CFE6FFDACFE6FF3FC1E6FF40C1B7
:1071A000E6FFF0EC28F0E106E106E106E106D9CFC2
:1071B000E6FFDACFE6FF73EC2AF0E552E552810EE6
:1071C000E66E030EE66E28EC2AF0E552E552D9CFC2
:1071D000E6FFDACFE6FF3DC1E6FF3EC1E6FFF0EC99
:1071E00028F0E106E106E106E106D9CFE6FFDACFB5
:1071F000E6FF73EC2AF0E552E552000EE66E030E50
:10720000E66E28EC2AF0E552E552D9CFE6FFDACF58
:10721000E6FF38C1E6FF39C1E6FFF0EC28F0E106F1
:10722000E106E106E106D9CFE6FFDACFE6FF73EC2F
:107230002AF0E552E552A10EE66E030EE66E28EC4A
:107240002AF0E552E552D9CFE6FFDACFE6FF010199
:1072500038514825006E39514921016E00C0E6FFC2
:1072600001C0E6FFF0EC28F0E106E106E106E106E8
:10727000D9CFE6FFDACFE6FF73EC2AF0E552E5520C
:10728000B00EE66E030EE66E28EC2AF0E552E552EB
:10729000D9CFE6FFDACFE6FF010138513F25026E74
:1072A00039514021036E02504825006E0350492198
:1072B000016E00C0E6FF01C0E6FFF0EC28F0E10639
:1072C000E106E106E106D9CFE6FFDACFE6FF73EC8F
:1072D0002AF0E552E552730EE66E030EE66E28ECD8
:1072E0002AF0E552E552D9CFE6FFDACFE6FF41C1F9
:1072F000E6FF42C1E6FFF0EC28F0E106E106E10618
:10730000E106D9CFE6FFDACFE6FF73EC2AF0E552CB
:10731000E552930EE66E030EE66E28EC2AF0E55277
:10732000E552D9CFE6FFDACFE6FF43C1E6FF44C11D
:10733000E6FFF0EC28F0E106E106E106E106D9CF30
:10734000E6FFDACFE6FF73EC2AF0E552E552D9CF3B
:10735000E1FFE552E7CFD9FF120001010D910E6B5D
:107360001200D9CFE6FFE1CFD9FF070EE12684A6B0
:1073700011D001010DA10CD00D918588E00EE66EB3
:10738000040EE66E28EC2AF0E552E552F6EC21F008
:10739000DF6A4ED101010DB1FFD00D818598D10E6C
:1073A000E66E040EE66E28EC2AF0E552E55280EC1B
:1073B00035F001014A5102E0F4EC21F0010EDB6AE4
:1073C00004010E510F1125E1200EF36E010EDBCFEB
:1073D000F4FFF350F45C1DE2010EDB500101016A81
:1073E0004125006E4251012200C0E6FF01C0E6FFC8
:1073F000F30EE66E040EE66EA6EC48F0E106E1063A
:10740000E106E106F3CF0EF4F4CF0FF4010EDB2A10
:10741000D7D70E510F1101E07ED041C1E6FF42C126
:10742000E6FF010EE66E000EE66EE66AF30EE66E0D
:10743000040EE66E4EEC40F0F56E070EE15EF55080
:10744000010EDB6A100EF36E010EDBCFF4FFF3507A
:10745000F45C0BE2010EDB50EA6A4D0FE96E010E9F
:10746000EA22EF6A010EDB2AEDD7020EDB6A030E79
:10747000DB6A020EDBCF00F0030EDBCF01F0400E23
:1074800001014703F350026E036A0250005C03508F
:10749000015816E2100EE66EE66A4D0EE66E010E1B
:1074A000E66E000EE66EE66A6AEC45F0F56E060ED4
:1074B000E15EF550020EDB2A030E01E3DB2AD9D789
:1074C000010EDB6A04010E510F1125E1200EF36E4F
:1074D000010EDBCFF4FFF350F45C1DE2010EDB5034
:1074E0000101016A4125006E4251012200C0E6FF00
:1074F00001C0E6FFF30EE66E040EE66EA6EC48F061
:10750000E106E106E106E106F3CF0EF4F4CF0FF455
:10751000010EDB2AD7D70EC4E6FF0FC4E6FF75ECD9
:107520004BF0E552E552040EF3CFDBFF050EF4CF2E
:10753000DBFF010EE66E010EE66E6CEC33F0E552F9
:10754000E552B3EC51F0E76E060EE7CFDBFFDB5000
:1075500020E1040EDBCF00F0050EDBCF01F00101CE
:107560004351005C4451015814E3040EDBCFE6FFA5
:10757000050EDBCFE6FFE66A000EE66EE66A010E58
:10758000E66E010EE66E4EEC40F0F56E070EE15E23
:10759000F55045EC4AF04BD0435104010E5D01011A
:1075A000445104010F5902E2000E01D0010E006E99
:1075B0000101000502E0000E01D0010E001437E0C9
:1075C000006B0EC4E6FF0FC4E6FF75EC4BF0E5520E
:1075D000E552040EF3CFDBFF050EF4CFDBFF040E04
:1075E000DBCF00F0050EDBCF01F001014351005C61
:1075F000445101581CE3010EE66E010EE66E6CEC80
:1076000033F0E552E552040EDBCFE6FF050EDBCF8B
:10761000E6FFE66A000EE66EE66A010EE66E010E11
:10762000E66E4EEC40F0F56E070EE15EF550DF6859
:10763000DF5000D0D9CFE1FFE552E7CFD9FF1200EC
:10764000D9CFE6FFE1CFD9FF000EE66E050EE66E5C
:10765000E66A010EE66EFD0EDBCFE6FFFE0EDBCF27
:10766000E6FF81EC2EF0F56E060EE15EF550000EA1
:10767000E66E060EE66EE66A010EE66E08EC2FF088
:10768000E106E106E106E106E552E7CFD9FF120087
:10769000D9CFE6FFE1CFD9FF000EE66E050EE66E0C
:1076A000E66A010EE66EFD0EDBCFE6FFFE0EDBCFD7
:1076B000E6FF4EEC2FF0F56E060EE15EF550000E83
:1076C000E66E060EE66EE66A010EE66ED4EC2FF06C
:1076D000E106E106E106E106E552E7CFD9FF120037
:1076E000D9CFE6FFE1CFD9FFCC0EE66E020EE66EF3
:1076F000EC0EE66E040EE66EFD0EDBCF02F0FE0E23
:10770000DBCF03F00350020AE8AE02D0D89004D0D9
:10771000000E025C020E035802E2000E01D0010EC0
:10772000006E016A00BE016800C0E6FF01C0E6FF0E
:107730002AEC23F0F56E060EE15EF550FD0EDBCF70
:1077400000F0FE0EDBCF01F00150010AE8AE02D0DE
:10775000D89004D0000E005C010E01580CE2FD0E22
:10776000DBCFE9FFFE0EDBCFEAFF000EE926050EB8
:10777000EA22EF5010D0FD0EDBCFE9FFFE0EDBCF8B
:10778000EAFF000EE95E010EEA5A000EE926060E37
:10779000EA22EF5000D0E552E7CFD9FF1200D9CF4F
:1077A000E6FFE1CFD9FF020EE126E00EE66E020E03
:1077B000E66EEC0EE66E040EE66EFD0EDBCF02F01A
:1077C000FE0EDBCF03F00350020AE8AE02D0D890E1
:1077D00004D0000E025C020E035802E2000E01D03B
:1077E000010E006E016A00BE016800C0E6FF01C024
:1077F000E6FF2AEC23F0F56E060EE15EF550E10E91
:10780000E66E020EE66EEC0EE66E040EE66E010EFD
:10781000E76EFD0EDBCF00F0FE0EDBCF01F0E75090
:107820000016016A00C0E6FF01C0E6FF2AEC23F063
:10783000F56E060EE15EF550FD0EDB2AFE0E01E34D
:10784000DB2AFD0EDBCF00F0FE0EDBCF01F0015096
:10785000010AE8AE02D0D89004D0000E005C010E00
:10786000015838E2FD0EDBCFE9FFFE0EDBCFEAFF69
:10787000000EE926050EEA22EF50DE6EDD6ADECF4D
:1078800000F0DDCF01F000C001F0006A00C0DEFFB3
:1078900001C0DDFFFD0EDB06FE0E01E2DB06FD0E84
:1078A000DBCFE9FFFE0EDBCFEAFF000EE926050E77
:1078B000EA22EF50E76E000EDFCF00F0010EDBCFC3
:1078C00001F0E7500026000E012200C0DEFF01C0DB
:1078D000DDFF47D0FD0EDBCF00F0FE0EDBCF01F069
:1078E000000E005E010E015AFD0E00C0DBFFFE0E11
:1078F00001C0DBFFFD0EDBCFE9FFFE0EDBCFEAFFB1
:10790000000EE926060EEA22EF50DE6EDD6ADECFBB
:1079100000F0DDCF01F000C001F0006A00C0DEFF22
:1079200001C0DDFFFD0EDB06FE0E01E2DB06FD0EF3
:10793000DBCFE9FFFE0EDBCFEAFF000EE926060EE5
:10794000EA22EF50E76E000EDFCF00F0010EDBCF32
:1079500001F0E7500026000E012200C0DEFF01C04A
:10796000DDFFDECF00F0DDCF01F000C0F3FF01C08E
:10797000F4FF00D0D9CFE1FFE552E7CFD9FF1200E5
:10798000D9CFE6FFE1CFD9FFFA0EE66E020EE66E22
:10799000EC0EE66E040EE66EFD0EDBCF02F0FE0E80
:1079A000DBCF03F00350020AE8AE02D0D89004D037
:1079B000000E025C020E035802E2000E01D0010E1E
:1079C000006E016A00BE016800C0E6FF01C0E6FF6C
:1079D0002AEC23F0F56E060EE15EF550FD0EDBCFCE
:1079E00000F0FE0EDBCF01F00150010AE8AE02D03C
:1079F000D89004D0000E005C010E01580EE2FD0E7E
:107A0000DBCFE9FFFE0EDBCFEAFF000EE926050E15
:107A1000EA22FC0EDBCFEFFF11D0FD0EDBCFE9FF3A
:107A2000FE0EDBCFEAFF000EE95E010EEA5A000E01
:107A3000E926060EEA22FC0EDBCFEFFFE552E7CF88
:107A4000D9FF1200D9CFE6FFE1CFD9FF020EE12620
:107A50000E0EE66E030EE66EEC0EE66E040EE66E9D
:107A6000FD0EDBCF02F0FE0EDBCF03F00350020A67
:107A7000E8AE02D0D89004D0000E025C020E03588B
:107A800002E2000E01D0010E006E016A00BE016824
:107A900000C0E6FF01C0E6FF2AEC23F0F56E060EFB
:107AA000E15EF5500F0EE66E030EE66EEC0EE66E2E
:107AB000040EE66E010EE76EFD0EDBCF00F0FE0E4B
:107AC000DBCF01F0E7500016016A00C0E6FF01C0FD
:107AD000E6FF2AEC23F0F56E060EE15EF550FD0E92
:107AE000DBCF00F0FE0EDBCF01F00150010AE8AE63
:107AF00002D0D89004D0000E005C010E015834E290
:107B0000FF0EE76EFB0EDBCF00F0FC0EDBCF01F0CB
:107B1000E7500016016AFD0EDBCFE9FFDB2AFE0EFF
:107B2000DBCFEAFF01E3DB2A000EE926050EEA229D
:107B300000C0EFFFFB0EDBCF00F0FC0EDBCF01F04F
:107B4000000E0016FF0E011601C000F0016AFD0EC6
:107B5000DBCFE9FFFE0EDBCFEAFF000EE926050EC4
:107B6000EA2200C0EFFF3BD0D950FD0FE96EFF0EB7
:107B7000DA20EA6EEE52ED06FF0EE76EFB0EDBCF6B
:107B800000F0FC0EDBCF01F0E7500016016AFD0E9D
:107B9000DBCFE9FFDB2AFE0EDBCFEAFF01E3DB2AC6
:107BA000000EE926060EEA2200C0EFFFFB0EDBCF37
:107BB00000F0FC0EDBCF01F0000E0016FF0E0116E8
:107BC00001C000F0016AFD0EDBCFE9FFFE0EDBCF46
:107BD000EAFF000EE926060EEA2200C0EFFFD9CF29
:107BE000E1FFE552E7CFD9FF1200D9CFE6FFE1CFA1
:107BF000D9FF070EE1260B0EF36E020EF3CFDBFF6B
:107C0000030EDB6ADE68DD68040EDB6A050EDB6AE4
:107C1000020EDBCF00F0030EDBCF01F00150020AB1
:107C2000E8AE02D0D89004D0000E005C020E0158DD
:107C300058E2DECF02F0DDCF03F00001800E031525
:107C400050E0020EDBCFE6FF030EDBCFE6FF48DDA0
:107C5000E552E552E76E060EE7CFDBFFDB500F087B
:107C600031E0D950020FE96EDACFEAFF0B0EEE5E7B
:107C7000000EED5A020EDBCFE6FF030EDBCFE6FF70
:107C80002FDDE552E552E76E060EE7CFDBFFDB5056
:107C900004E0060EDB50E50806E1040EDBCFDEFF54
:107CA000DBCFDDFF0ED0D950020FE96EDACFEAFF4D
:107CB0002B0EEE26000EED22040EDB2A050E01E34C
:107CC000DB2A0ED0D950020FE96EDACFEAFF200E80
:107CD000EE26000EED22040EDB2A050E01E3DB2A60
:107CE00097D7DECF00F0DDCF01F000C0F3FF01C079
:107CF000F4FF00D0D9CFE1FFE552E7CFD9FF120062
:107D0000D9CFE6FFE1CFD9FF040EE126A9EC30F090
:107D100005EC31F0000165390F0B0A0DF350DE6EF2
:107D2000DD6A0F0E6515DE26000EDD22D9CFE9FFD4
:107D3000DACFEAFF020EEECFDBFF030EEDCFDBFF63
:107D4000D950020FE96EDACFEAFF0B0ED890EE366B
:107D5000ED36E806FBE1000164390F0B0A0DF35024
:107D6000DE6EDD6A0F0E6415DE26000EDD22DECF2C
:107D700000F0DDCF01F0050ED89000360136E804A2
:107D8000FBE1D950020FE96EDACFEAFF0050EE2690
:107D90000150ED22020EDBCF00F0030EDBCF01F02D
:107DA00000C0F3FF01C0F4FF00D0D9CFE1FFE552DE
:107DB000E7CFD9FF1200D9CFE6FFE1CFD9FF040EFC
:107DC000E126A9EC30F005EC31F0000169390F0B28
:107DD0000A0DF350DE6EDD6A0F0E6915DE26000E09
:107DE000DD22140EDE26000EDD22DECF00F0DDCF18
:107DF00001F000C001F0006AD8900136020E00C008
:107E0000DBFF030E01C0DBFF68390F0B010B0A0D0E
:107E1000F350DE6EDD6A0F0E6815DE26000EDD22E1
:107E2000DECF00F0DDCF01F0050ED8900036013630
:107E3000E804FBE1D950020FE96EDACFEAFF005007
:107E4000EE260150ED22000167390F0B0A0DF350A9
:107E5000DE6EDD6A0F0E6715DE26000EDD22DECF38
:107E600000F0DDCF01F0D950020FE96EDACFEAFF62
:107E70000050EE260150ED22020EDBCF00F0030E83
:107E8000DBCF01F000C0F3FF01C0F4FF00D0D9CF79
:107E9000E1FFE552E7CFD9FF1200D9CFE6FFE1CFEE
:107EA000D9FF070EE126000E01011915006EFF0E25
:107EB0001A15016E050E00C0DBFF060E01C0DBFFC8
:107EC000D950050FE96EDACFEAFF040E0F0B06E07A
:107ED000EC52D890ED32EF32E806FAE1D950050FB6
:107EE000E96EDACFEAFF040E0F0B06E0EC52D890F1
:107EF000ED32EF32E806FAE1D950050FE96EDACF3C
:107F0000EAFF01014851EE264951ED22050EDB50F2
:107F100038250001006F060EDB50010139210001F8
:107F2000016F00C0E6FF01C0E6FF20EC3BF0E55228
:107F3000E552040EDE6EDD6ADECFE6FFDDCFE6FF42
:107F40002EDCE552E552020EF3CFDBFF030EF4CF39
:107F5000DBFF040EDB6AD950020FE96EDACFEAFFCD
:107F6000EE50ED1059E0040EDB5056E1020EDE2615
:107F7000000EDD22DECF00F0DDCF01F0005C020E4E
:107F800001580FE2DECFE6FFDDCFE6FFCFEC3BF09E
:107F9000E552E552020EF3CFDBFF030EF4CFDBFF19
:107FA0003AD0050EDBCF00F0060EDBCF01F0010169
:107FB00000503F5D0150405929E3050EDB2A060EB3
:107FC00001E3DB2A050EDB5038250001006F060EA9
:107FD000DB50010139210001016F00C0E6FF01C043
:107FE000E6FF20EC3BF0E552E552DE6ADD6ADECFCB
:107FF000E6FFDDCFE6FFCFEC3BF0E552E552020EA7
:10800000F3CFDBFF030EF4CFDBFF05D0010EF36EE1
:10801000040EF3CFDBFF9FD7040EDB5036E1050ED5
:10802000DBCF00F0060EDBCF01F00006000E015A98
:10803000040ED89000360136E804FBE1FD0EDBCFDC
:10804000E9FFFE0EDBCFEAFF00C0EEFF01C0EDFF4F
:10805000FD0EDBCFE9FFFE0EDBCFEAFF040ED8906A
:10806000EE36ED36E806FBE1DECF00F0DDCF01F0C5
:10807000D89001320032FD0EDBCFE9FFFE0EDBCFE0
:10808000EAFF0050EE260150ED22040EDB5000D036
:10809000D9CFE1FFE552E7CFD9FF1200D9CFE6FFF4
:1080A000E1CFD9FF0F0EE126B1EC39F0000901E173
:1080B0004DD201014A5101E143D2020EDB6A030EA7
:1080C000DB68040EDB68F80EDBCF00F0F90EDBCFC7
:1080D00001F04151001802E14251011838E1020E4D
:1080E000DBCF00F001013D51005C000E3E552EE259
:1080F000030EDBCF01F0040EDBCF02F00001800E97
:10810000021524E0020EDB500101016A4125006ED8
:108110004251012200C0E6FF01C0E6FF20EC3BF027
:10812000E552E55262DD030EF3CFDBFF040EF4CF20
:10813000DBFF030EDBCF00F0040EDBCF01F000010C
:10814000800E011502E0020EDB2AC9D711D0F80E0D
:10815000DBCFE6FFF90EDBCFE6FF20EC3BF0E5528C
:10816000E55243DD030EF3CFDBFF040EF4CFDBFF5C
:10817000030EDBCF00F0040EDBCF01F00001800E18
:10818000011501E0D6D1020EDB5001010F6F106B1B
:10819000030EDBCF11F1040EDBCF12F1176B186B5E
:1081A000196B1A6B136B146B156B166B200E0F6E1D
:1081B000106A030EDBCF14F0040EDBCF15F079EC60
:1081C00023F0070E0DC0DBFF080E0EC0DBFF050E0F
:1081D000DB6A060EDB6AFD0EDBCFE9FFFE0EDBCFAE
:1081E000EAFFEF502CE0FD0EDBCFE9FFFE0EDBCF08
:1081F000EAFFEF502E0823E0FD0EDBCFE9FFFE0E75
:10820000DBCFEAFFEF50E66E070EDBCFE6FF080E8E
:10821000DBCFE6FFC0EC3CF0E106E106E106070E2D
:10822000DB2A080E01E3DB2AFD0EDB2AFE0E01E34A
:10823000DB2A050EDB2A060E01E3DB2ACCD7050E6E
:10824000DBCF00F0060EDBCF01F0080E005C000E65
:10825000015818E2200EE66E070EDBCFE6FF080E8F
:10826000DBCFE6FFC0EC3CF0E106E106E106070EDD
:10827000DB2A080E01E3DB2A050EDB2A060E01E3EA
:10828000DB2ADDD7FD0EDBCFE9FFFE0EDBCFEAFFF9
:10829000EF502E0862E1FD0EDB2AFE0E01E3DB2A21
:1082A000050EDB6A060EDB6AFD0EDBCFE9FFFE0E74
:1082B000DBCFEAFFEF502EE0050EDBCF00F0060E1D
:1082C000DBCF01F0030E005C000E015823E2FD0E2F
:1082D000DBCFE9FFFE0EDBCFEAFFEF50E66E070EC5
:1082E000DBCFE6FF080EDBCFE6FFC0EC3CF0E1069B
:1082F000E106E106070EDB2A080E01E3DB2AFD0E8C
:10830000DB2AFE0E01E3DB2A050EDB2A060E01E363
:10831000DB2ACAD7050EDBCF00F0060EDBCF01F05B
:10832000030E005C000E015818E2200EE66E070EE8
:10833000DBCFE6FF080EDBCFE6FFC0EC3CF0E1064A
:10834000E106E106070EDB2A080E01E3DB2A050E33
:10835000DB2A060E01E3DB2ADDD7FA0EDB5000082C
:1083600013E2100EE66E070EDBCFE6FF080EDBCF42
:10837000E6FFC0EC3CF0E106E106E106070EDB2A71
:10838000080E01E3DB2A11D0E66A070EDBCFE6FF19
:10839000080EDBCFE6FFC0EC3CF0E106E106E106AB
:1083A000070EDB2A080E01E3DB2A050EDB6A060E48
:1083B000DB6A050EDBCF00F0060EDBCF01F00A0E04
:1083C000005C000E015817E2E66A070EDBCFE6FFFD
:1083D000080EDBCFE6FFC0EC3CF0E106E106E1066B
:1083E000070EDB2A080E01E3DB2A050EDB2A060E48
:1083F00001E3DB2ADED784DC090EF3CFDBFF0A0EB4
:10840000F4CFDBFF090EDBCFE6FF0A0EDBCFE6FF82
:10841000070EDBCFE6FF080EDBCFE6FF22EC3DF0D8
:10842000E106E106E106E106D950070FE96EDACF71
:10843000EAFF020EEE26000EED22BDDC090EF3CFA0
:10844000DBFF0A0EF4CFDBFF090EDBCFE6FF0A0EDF
:10845000DBCFE6FF070EDBCFE6FF080EDBCFE6FF44
:1084600022EC3DF0E106E106E106E106D950070FF6
:10847000E96EDACFEAFF020EEE26000EED22050EBF
:10848000DB6A060EDB6A050EDBCF00F0060EDBCFE3
:1084900001F0005C000E015817E2E66A070EDBCF20
:1084A000E6FF080EDBCFE6FFC0EC3CF0E106E1069C
:1084B000E106070EDB2A080E01E3DB2A050EDB2AA4
:1084C000060E01E3DB2ADFD7F80EDBCF00F0F90E52
:1084D000DBCF01F001014151001802E142510118C6
:1084E00010E1020EDB50016A4125006E425101226B
:1084F00000C0E6FF01C0E6FF48EC3BF0E552E55264
:108500000AD0F80EDBCFE6FFF90EDBCFE6FF48EC32
:108510003BF0E552E552F80EDBCF20F1F90EDBCF50
:1085200021F10101010E0E6FDE6ADD6A4B6B4C6BAF
:1085300006D0DE68DD6801019A0E4B6F4C6905D0EC
:10854000DE68DD689B0E4B6F4C6906D0DE68DD6827
:1085500001019C0E4B6F4C69DECF00F0DDCF01F0C6
:1085600000C0F3FF01C0F4FF00D0D9CFE1FFE55216
:10857000E7CFD9FF1200D9CFE6FFE1CFD9FF020E36
:10858000E1260101000ED8801955000E1A5501E3AD
:1085900002D12B0EE66EEDEC29F0E55219C1E6FF93
:1085A0001AC1E6FF48EC2AF0E552E5522C0EE66EC1
:1085B000EDEC29F0E552000E01011915046EFF0ED5
:1085C0001A15056E05C004F0056A38510424026EC0
:1085D00039510520036E02504825006E0350492191
:1085E000016E00C0DEFF01C0DDFFDECFE6FFDDCFA4
:1085F000E6FF20EC3BF0E552E552E668E668FF0E48
:1086000001011915006E016AD8900036013600C0CC
:10861000E6FF01C0E6FF22EC3DF0E106E106E106DF
:10862000E106DECFE6FFDDCFE6FF48EC3BF0E552AA
:10863000E552DE5001013F250001006FDD500101D0
:1086400040210001016F00C0E6FF01C0E6FF48ECD9
:108650003BF0E552E55201011751181140E1640E5B
:10866000E66EEDEC29F0E552010120510F25006E78
:1086700021511021016E00C0E6FF01C0E6FF20EC91
:108680003BF0E552E55219C1E6FF1AC1E6FF11C100
:1086900000F012C101F0050ED89000360136E80650
:1086A000FBE11A0E0026000E012200C0E6FF01C009
:1086B000E6FF22EC3DF0E106E106E106E1060101FC
:1086C00020510F25006E21511021016E00C0E6FFE0
:1086D00001C0E6FF48EC3BF0E552E5525AD017C125
:1086E000E6FF18C1E6FF48EC2AF0E552E552000E1D
:1086F00001011715046EFF0E1815056E05C004F074
:10870000056A38510424026E39510520036E025067
:108710004825006E03504921016E00C0DEFF01C0F4
:10872000DDFFDECFE6FFDDCFE6FF20EC3BF0E552DC
:10873000E55219C1E6FF1AC1E6FFFF0E0101171548
:10874000006E016AD8900036013600C0E6FF01C015
:10875000E6FF22EC3DF0E106E106E106E106DECFB0
:10876000E6FFDDCFE6FF48EC3BF0E552E552DE5098
:1087700001013F250001006FDD5001014021000192
:10878000016F00C0E6FF01C0E6FF48EC3BF0E55298
:10879000E5526AEC2AF0D9CFE1FFE552E7CFD9FFE5
:1087A0001200D9CFE6FFE1CFD9FF060EE126010185
:1087B00020510F25006E21511021016E00C0E6FFEF
:1087C00001C0E6FF20EC3BF0E552E55211C104F098
:1087D00012C105F0050ED89004360536E806FBE117
:1087E0001E0E0426000E052204C0E6FF05C0E6FFAB
:1087F000CFEC3BF0E552E552F3CF00F0F4CF01F0BF
:10880000026A036A00C0DFFF010E01C0DBFF020E37
:1088100002C0DBFF030E03C0DBFFD9CFE9FFDACFD5
:10882000EAFF040EE76ED890000EEF36010EEB362D
:10883000020EEB36030EEB36E706F5E1D9CFE9FF82
:10884000DACFEAFF040EE76ED890000EEF36010E85
:10885000EB36020EEB36030EEB36E706F5E1D9CF29
:10886000E9FFDACFEAFF040EE76ED890000EEF368C
:10887000010EEB36020EEB36030EEB36E706F5E1A2
:10888000D9CFE9FFDACFEAFF040EE76ED890000EE9
:10889000EF36010EEB36020EEB36030EEB36E70633
:1088A000F5E111C100F012C101F0050ED8900036BB
:1088B0000136E806FBE11C0E0026000E012200C076
:1088C000E6FF01C0E6FFCFEC3BF0E552E552040EB7
:1088D000F3CFDBFF050EF4CFDBFF040EDBCF04F09C
:1088E000050EDBCF05F0066A076AD9CFE9FFDACFBC
:1088F000EAFFEE500424006EEE500520016EEE50AB
:108900000620026EEE500720036E00C0DFFF010E4E
:1089100001C0DBFF020E02C0DBFF030E03C0DBFF62
:10892000FD0EDBCF04F0FE0EDBCF05F0066A076A12
:10893000D9CFE9FFDACFEAFFEE500424006EEE5003
:108940000520016EEE500620026EEE500720036EE9
:1089500000C0DFFF010E01C0DBFF020E02C0DBFF23
:10896000030E03C0DBFFD9CFE9FFDACFEAFFEECF7A
:1089700000F0EECF01F0EECF02F0EFCF03F0026A8D
:10898000036A040E00C0DBFF050E01C0DBFF040E0E
:10899000DBCFE6FF050EDBCFE6FF11C100F012C111
:1089A00001F0D89000360136E806FBE11C0E0026E7
:1089B000000E012200C0E6FF01C0E6FF22EC3DF000
:1089C000E106E106E106E106D9CFE9FFDACFEAFFE9
:1089D000040EE76ED890030EEB32020EEB32010E5E
:1089E000EB32EF32E706F6E1D9CFE9FFDACFEAFF63
:1089F000040EE76ED890030EEB32020EEB32010E3E
:108A0000EB32EF32E706F6E1D9CFE9FFDACFEAFF42
:108A1000040EE76ED890030EEB32020EEB32010E1D
:108A2000EB32EF32E706F6E1D9CFE9FFDACFEAFF22
:108A3000040EE76ED890030EEB32020EEB32010EFD
:108A4000EB32EF32E706F6E1D9CFE9FFDACFEAFF02
:108A5000EECF00F0EECF01F0EECF02F0EFCF03F05B
:108A6000026A036A040E00C0DBFF050E01C0DBFFD3
:108A7000040EDBCFE6FF050EDBCFE6FF11C100F0F1
:108A800012C101F0D89000360136E806FBE11E0E57
:108A90000026000E012200C0E6FF01C0E6FF22EC26
:108AA0003DF0E106E106E106E106010120510F2556
:108AB000006E21511021016E00C0E6FF01C0E6FFEB
:108AC00048EC3BF0E552E552D9CFE1FFE552E7CF64
:108AD000D9FF1200D9CFE6FFE1CFD9FF040EE1267E
:108AE000DE6ADD6A01010E0501E03AD119511A1161
:108AF0001DE1190EE66E010EE66E4DEC3FF0E552FB
:108B0000E552000807E2DE68DD680101990E4B6F4F
:108B10004C690CD019C1E6FF1AC1E6FF48EC2AF0F7
:108B2000E552E55201011B6B1C6B1D6BDECF00F0A3
:108B3000DDCF01F00001800E011501E0FBD0010145
:108B40004751046E056A19C102F01AC103F0020E02
:108B5000025E000E035A02C00FF003C010F004C002
:108B600014F005C015F0A6EC23F00D5001014325CB
:108B7000006E0E504421016E1B511F6B00241E6FAE
:108B800001501F23400EE66EEDEC29F0E5521EC1A8
:108B9000E6FF1FC1E6FF48EC2AF0E552E5521EC190
:108BA000E6FF1FC1E6FF20EC3BF0E552E552F90E6F
:108BB000DBCF0FF0FA0EDBCF10F0020E0FC0DBFFA1
:108BC000030E10C0DBFFD950020FE96EDACFEAFFC7
:108BD000EE50ED1001E196D00101000E1C5D020E79
:108BE0001D5970E31EC1E6FF1FC1E6FF48EC3BF0D4
:108BF000E552E55201011B2B47511B5D06E21E2B7E
:108C0000000E1F231C6B1D6B5CD0190EE66E010E4F
:108C1000E66E4DEC3FF0E552E552000817E2020E19
:108C2000DB6A030EDB6A020EDBCF0FF0030EDBCF35
:108C300010F0F90E0FC0DBFFFA0E10C0DBFFDE688C
:108C4000DD680101990E4B6F4C693BD019C1E6FFFD
:108C50001AC1E6FF48EC2AF0E552E55201011B6B10
:108C60001C6B1D6B4751046E056A19C102F01AC1D5
:108C700003F0020E025E000E035A02C00FF003C0A2
:108C800010F004C014F005C015F0A6EC23F00D5050
:108C900001014325006E0E504421016E1B511F6BD4
:108CA00000241E6F01501F23400EE66EEDEC29F0EC
:108CB000E5521EC1E6FF1FC1E6FF48EC2AF0E5526F
:108CC000E5521FD0FB0EDBCFE9FFFC0EDBCFEAFF46
:108CD000EF50E66E1CC1E6FF1DC1E6FFC0EC3CF0A4
:108CE000E106E106E10601011C2B000E1D23FB0E2F
:108CF000DB2AFC0E01E3DB2A020EDB06030E01E297
:108D0000DB0661D70101000E1C5D020E1D590AE24F
:108D1000E66A1CC1E6FF1DC1E6FFC0EC3CF0E106BF
:108D2000E106E1061EC1E6FF1FC1E6FF48EC3BF08D
:108D3000E552E55201011951171902E11A511819AA
:108D400005E019DC19C117F11AC118F1F90EDBCFD2
:108D5000E6FFFA0EDBCFE6FF24DDE552E55205D053
:108D6000DE68DD68380E4B6F4C69DECF00F0DDCF7A
:108D700001F000C0F3FF01C0F4FF00D0D9CFE1FF44
:108D8000E552E7CFD9FF1200D9CFE6FFE1CFD9FFF7
:108D9000020EE126DE6ADD6A01010E6B00D0D9CF3A
:108DA000E1FFE552E7CFD9FF1200D9CFE6FFE1CFCF
:108DB000D9FFFE0EDB380F0BF36EFE0EF3CFDBFF99
:108DC000DB5009080BE2370E006EFE0EDBCFE7FF2B
:108DD0000050E726FE0EE7CFDBFF0AD0300E006E14
:108DE000FE0EDBCFE7FF0050E726FE0EE7CFDBFFEE
:108DF000FE0EDBCFE6FFEDEC29F0E552E552E7CFC2
:108E0000D9FF1200D9CFE6FFE1CFD9FFFE0EDB98E4
:108E1000DB9ADB9CDB9EFE0EDB5009080BE2370E73
:108E2000006EFE0EDBCFE7FF0050E726FE0EE7CF19
:108E3000DBFF0AD0300E006EFE0EDBCFE7FF0050E6
:108E4000E726FE0EE7CFDBFFFE0EDBCFE6FFEDEC05
:108E500029F0E552E552E7CFD9FF1200D9CFE6FF5E
:108E6000E1CFD9FF030EE126FE0EDB50100DF350CB
:108E7000016A000F006E050E0122010E00C0DBFF2B
:108E8000020E01C0DBFFDF6A100EDF5C3AE2010E6A
:108E9000DBCFE9FF020EDBCFEAFFEF50E66E85DFA6
:108EA000E552010EDBCFE9FF020EDBCFEAFFEF5008
:108EB000E66EA8DFE552010EDB2A020E01E3DB2A93
:108EC000010EDBCFE9FF020EDBCFEAFFEF50E66ECB
:108ED0006CDFE552010EDBCFE9FF020EDBCFEAFFCC
:108EE000EF50E66E8FDFE552010EDB2A020E01E342
:108EF000DB2A200EE66EEDEC29F0E552020EDF26AD
:108F0000C3D7FE0EDB50100DF350016A000F006E48
:108F1000050E0122010E00C0DBFF020E01C0DBFFC7
:108F2000DF6A100EDF5C2CE2010EDBCFE9FF020EE0
:108F3000DBCFEAFFEFCF00F0200E005C15E3010E5F
:108F4000DBCFE9FF020EDBCFEAFFEF507E080CE338
:108F5000010EDBCFE9FF020EDBCFEAFFEF50E66E3A
:108F6000EDEC29F0E55205D02E0EE66EEDEC29F081
:108F7000E552010EDB2A020E01E3DB2ADF2AD1D7FC
:108F80000D0EE66EEDEC29F0E5520A0EE66EEDEC04
:108F900029F0E552D9CFE1FFE552E7CFD9FF120022
:108FA000D9CFE6FFE1CFD9FF030EE126FE0EDB505D
:108FB000100DF350016A000F006E060E0122010E23
:108FC00000C0DBFF020E01C0DBFFDF6A100EDF5CBA
:108FD0003AE2010EDBCFE9FF020EDBCFEAFFEF50F2
:108FE000E66EE3DEE552010EDBCFE9FF020EDBCFDA
:108FF000EAFFEF50E66E06DFE552010EDB2A020EB5
:1090000001E3DB2A010EDBCFE9FF020EDBCFEAFF33
:10901000EF50E66ECADEE552010EDBCFE9FF020E2D
:10902000DBCFEAFFEF50E66EEDDEE552010EDB2A04
:10903000020E01E3DB2A200EE66EEDEC29F0E5528C
:10904000020EDF26C3D7FE0EDB50100DF350016A6F
:10905000000F006E060E0122010E00C0DBFF020EA3
:1090600001C0DBFFDF6A100EDF5C2CE2010EDBCFFC
:10907000E9FF020EDBCFEAFFEFCF00F0200E005C2D
:1090800015E3010EDBCFE9FF020EDBCFEAFFEF5065
:109090007E080CE3010EDBCFE9FF020EDBCFEAFF17
:1090A000EF50E66EEDEC29F0E55205D02E0EE66E9F
:1090B000EDEC29F0E552010EDB2A020E01E3DB2A7A
:1090C000DF2AD1D70D0EE66EEDEC29F0E5520A0E3F
:1090D000E66EEDEC29F0E552D9CFE1FFE552E7CF9E
:1090E000D9FF1200D9CFE6FFE1CFD9FFE652FD0E3E
:1090F000DBCFE6FFFE0EDBCFE6FF20EC3BF0E552D8
:10910000E552DF6A100EDF5C06E2DFCFE6FFA6DE87
:10911000E552DF2AF7D7DF6A100EDF5C06E2DFCF09
:10912000E6FF3EDFE552DF2AF7D7E552E552E7CF0B
:10913000D9FF120041C1F3FF42C1F4FF00D0120079
:1091400043C1F3FF44C1F4FF00D01200D9CFE6FFC2
:10915000E1CFD9FF090EE126030EDB6A040EDB6ABC
:10916000070EDB6AFB0EDBCFE6FFFC0EDBCFE6FF74
:1091700020EC3BF0E552E552DF6A010EDB6A020E9D
:10918000DB6A010EDBCF00F0020EDBCF01F0FF0E39
:10919000005C000E01583AE2070EDB0437E0010ED6
:1091A000DBCFE9FF020EDBCFEAFF000EE926050E5A
:1091B000EA22EFCF00F0DF50E76EFD0EDBCFE9FFD4
:1091C000FE0EDBCFEAFFE750E926000EEA22EF5061
:1091D000005C15E1010EDB2A020E01E3DB2ADF2A27
:1091E0000A0EDF5C0BE1010EF36E070EF3CFDBFF1F
:1091F000010EDB50E76E080EE7CFDBFFD0D7DF6A4A
:10920000010EDB2A020E01E3DB2ABBD7070EDB507F
:1092100001E0BCD0DF6A010EDB6A020EDB6A010EE0
:10922000DBCF00F0020EDBCF01F0FF0E005C000E82
:1092300001583AE2070EDB0437E0010EDBCFE9FF0D
:10924000020EDBCFEAFF000EE926060EEA22EFCF80
:1092500000F0DF50E76EFD0EDBCFE9FFFE0EDBCF47
:10926000EAFFE750E926000EEA22EF50005C15E124
:10927000010EDB2A020E01E3DB2ADF2A0A0EDF5C85
:109280000BE1010EF36E070EF3CFDBFF010EDB5097
:10929000E76E080EE7CFDBFFD0D7DF6A010EDB2ACF
:1092A000020E01E3DB2ABBD7070EDB506EE0080E8F
:1092B000DB50110FEA6A000FE96E060EEA22EF504A
:1092C000E66ED950030FE96EDACFEAFFE552E750B8
:1092D000EE6EED6A030EDBCF00F0040EDBCF01F083
:1092E00000C001F0006A050E00C0DBFF060E01C0E1
:1092F000DBFF080EDB50100FEA6A000FE96E060E66
:10930000EA22EF50E66ED950030FE96EDACFEAFF9A
:10931000E552E750EE6EED6A050EDBCF00F0060E6B
:10932000DBCF01F0D950030FE96EDACFEAFF00502E
:10933000EE260150ED22D950030FE96EDACFEAFF95
:10934000020EEE5E000EED5A01014751006E016AF9
:10935000D950030FE96EDACFEAFF00C014F001C064
:1093600015F0EECF0FF0EDCF10F0A6EC23F00DC00E
:10937000EEFF0EC0EDFFD950030FE96EDACFEAFF22
:1093800001014351EE264451ED226ED0080EDB5010
:10939000110FEA6A000FE96E050EEA22EF50E66E41
:1093A000D950030FE96EDACFEAFFE552E750EE6ECF
:1093B000ED6A030EDBCF00F0040EDBCF01F000C03E
:1093C00001F0006A050E00C0DBFF060E01C0DBFFE6
:1093D000080EDB50100FEA6A000FE96E050EEA2254
:1093E000EF50E66ED950030FE96EDACFEAFFE5528F
:1093F000E750EE6EED6A050EDBCF00F0060EDBCF18
:1094000001F0D950030FE96EDACFEAFF0050EE26E3
:109410000150ED22D950030FE96EDACFEAFF020EB8
:10942000EE5E000EED5A01014751006E016AD950FF
:10943000030FE96EDACFEAFF00C014F001C015F0A7
:10944000EECF0FF0EDCF10F0A6EC23F00DC0EEFF45
:109450000EC0EDFFD950030FE96EDACFEAFF01012C
:109460004351EE264451ED22030EDBCF00F0040EF3
:10947000DBCF01F000C0F3FF01C0F4FF00D0D9CF73
:10948000E1FFE552E7CFD9FF1200D9CFE6FFE1CFE8
:10949000D9FF1B0EE126530EDF6EDE52590EDD6E34
:1094A000530EF36E020EF3CFDBFF540EF36E030E7A
:1094B000F3CFDBFF450EF36E040EF3CFDBFF4D0E53
:1094C000F36E050EF3CFDBFF200EF36E060EF3CF27
:1094D000DBFF200EF36E070EF3CFDBFF200EF36EE3
:1094E000080EF3CFDBFF200EF36E090EF3CFDBFF88
:1094F000200EF36E0A0EF3CFDBFF490EF36E0B0E58
:10950000F3CFDBFF4E0EF36E0C0EF3CFDBFF490EF5
:10951000F36E0D0EF3CFDBFF200EF36E0E0EF3CFC6
:10952000DBFF200EF36E0F0EF3CFDBFF200EF36E8A
:10953000100EF3CFDBFF200EF36E110EF3CFDBFF27
:10954000200EF36E120EF3CFDBFF540EF36E130EEC
:10955000F3CFDBFF580EF36E140EF3CFDBFF540E88
:10956000F36E150EF3CFDBFF160EDB6A170EDB6A08
:10957000180EDB6A190EDB6A1A0EDB6AD950170F58
:10958000E96EDACFEAFFEE50ED1026E1200EF36E21
:10959000160EDBCFF4FFF350F45C1EE2160EDB5028
:1095A0000101016A4125006E4251012200C0E6FF1F
:1095B00001C0E6FFD9CFE6FFDACFE6FFC7DDE1065F
:1095C000E106E106E106170EF3CFDBFF180EF4CF3C
:1095D000DBFF160EDB2AD2D7170EDBCFE6FF180E05
:1095E000DBCFE6FFD9500B0FE66EDACFE6FFAEDD3C
:1095F000E106E106E106E106190EF3CFDBFF1A0EE4
:10960000F4CFDBFFD950190FE96EDACFEAFFEE5045
:10961000ED100AE0190EDBCFE6FF1A0EDBCFE6FFF6
:1096200020EC3BF0E552E552430E0501005D1BE1E5
:10963000340E085D0AE199EC25F0010EE66E2F0E5E
:10964000E66E70EC25F0E552E552320E0501085D3C
:1096500009E199EC25F0E66A2F0EE66E70EC25F034
:10966000E552E55207D0E66A2F0EE66E70EC25F063
:10967000E552E552530E05010D5D2EE11A0EF36E13
:10968000160EF3CFDBFF0401006BDB50EA6A000F1C
:10969000E96E050EEA22EFCF00F0300E005C1BE30E
:1096A000160EDB50EA6A000FE96E050EEA22EF5053
:1096B000390811E30A0E0003F3CF00F4160EDB5055
:1096C000EA6A000FE96E050EEA22EF50D00F00277C
:1096D000160EDB2ADAD703D00401010E006FD9CFB2
:1096E000E1FFE552E7CFD9FF1200D9CFE6FFE1CF86
:1096F000D9FF110EE1260B0EDB6A0C0EDB6ADE6869
:10970000DD680F0EDB6A100EDB6ADECF00F0DDCF06
:1097100001F00001800E011539E00F0EDBCF02F0E1
:10972000100EDBCF03F001014751046E056A0450AF
:10973000025C055003582AE20F0EDBCF02F0100E38
:10974000DBCF03F0FD0EDB500224006EFE0EDB507B
:109750000320016E00C0E6FF01C0E6FF20EC3BF0F5
:10976000E552E552F5EC3DF0F3CFDEFFF4CFDDFF3F
:10977000DECF00F0DDCF01F00001800E011505E025
:109780000F0EDB2A100E01E3DB2ABFD7DECF00F07D
:10979000DDCF01F00001800E011501E1D2D1FD0EF7
:1097A000DBCF0FF0FE0EDBCF10F0010143510F5C59
:1097B000006E44511058016E0D0E00C0DBFF0E0EFE
:1097C00001C0DBFF4751006E016AD9500D0FE96EF1
:1097D000DACFEAFF00C014F001C015F0EECF0FF0B1
:1097E000EDCF10F00AEC22F00FC0EEFF10C0EDFF3D
:1097F000D9500D0FE96EDACFEAFF020EEE26000E09
:10980000ED220B0EDB6A0C0EDB6A01014751046E80
:10981000056AFD0EDBCF0FF0FE0EDBCF10F04351DB
:109820000F5C026E44511058036E02C00FF003C06B
:1098300010F004C014F005C015F00AEC22F00FC0BF
:1098400000F010C001F0020E0026000E0122040EEE
:1098500000C0DBFF050E01C0DBFF040EDBCFE6FF1F
:10986000050EDBCFE6FF4DEC37F0E552E552090E71
:10987000F3CFDBFF0A0EF4CFDBFFDECF00F0DDCF4E
:1098800001F00001800E011501E1AAD0D950090FA5
:10989000E96EDACFEAFF000ED880EE54000EED54E8
:1098A00001E39ED0040EDBCFE6FF050EDBCFE6FF23
:1098B0004DEC37F0E552E552090EF3CFDBFF0A0E0F
:1098C000F4CFDBFFD950090FE96EDACFEAFF000EC3
:1098D000D880EE54000EED5401E381D00F0EDB6A08
:1098E000100EDB6ADECF00F0DDCF01F00001800E4C
:1098F000011551E00F0EDBCF02F0100EDBCF03F0AD
:1099000001014751046E056A0450025C055003587A
:1099100042E24751066E076A090EDBCF04F00A0ED9
:10992000DBCF05F0020E045E000E055A04C00FF0F6
:1099300005C010F006C014F007C015F0A6EC23F027
:109940000D5001014325026E0E504421036E0F0E8F
:10995000DB500224006E100EDB500320016E00C0AD
:10996000E6FF01C0E6FF20EC3BF0E552E552F5ECE6
:109970003DF0F3CFDEFFF4CFDDFFDECF00F0DDCF33
:1099800001F00001800E011505E00F0EDB2A100E1C
:1099900001E3DB2AA7D7090EDBCF0FF00A0EDBCFDE
:1099A00010F00D0E0FC0DBFF0E0E10C0DBFF040E1B
:1099B000DBCF0FF0050EDBCF10F00B0E0FC0DBFF7F
:1099C0000C0E10C0DBFF090EDBCF0FF00A0EDBCF51
:1099D00010F0040E0FC0DBFF050E10C0DBFF4DD7EB
:1099E000DECF00F0DDCF01F0800E011501E17BD06C
:1099F0000D0EDBCF19F10E0EDBCF1AF10D0EDBCF02
:109A000017F10E0EDBCF18F141C120F142C121F157
:109A10000101010E0E6F47051B6F1C6B020E1D6FBF
:109A2000060EDB6A100EF36E060EDBCFF4FFF3506A
:109A3000F45C0BE2060EDB50EA6A4D0FE96E010E94
:109A4000EA22EF6A060EDB2AEDD7070EDB6A080E64
:109A5000DB6A070EDBCF00F0080EDBCF01F0200E33
:109A600001014703F350026E036A0250005C035089
:109A7000015816E2100EE66EE66A4D0EE66E010E15
:109A8000E66E000EE66EE66A6AEC45F0F56E060ECE
:109A9000E15EF550070EDB2A080E01E3DB2AD9D779
:109AA0004751046E056A17C102F018C103F0020E97
:109AB000025E000E035A02C00FF003C010F004C093
:109AC00014F005C015F0A6EC23F00D50010143255C
:109AD000006E0E504421016E020E00C0DBFF030E2B
:109AE00001C0DBFF2DD001014751066E076A090E48
:109AF000DBCF04F00A0EDBCF05F0020E045E000E91
:109B0000055A04C00FF005C010F006C014F007C0DD
:109B100015F0A6EC23F00D5001014325026E0E5006
:109B20004421036E0F0EDB500224006E100EDB503A
:109B30000320016E020E00C0DBFF030E01C0DBFF3D
:109B400014D00F0EDBCF02F0100EDBCF03F0FD0EB2
:109B5000DB500224006EFE0EDB500320016E020E6D
:109B600000C0DBFF030E01C0DBFF020EDBCF00F005
:109B7000030EDBCF01F000C0F3FF01C0F4FF00D003
:109B8000D9CFE1FFE552E7CFD9FF1200D9CFE6FFE9
:109B9000E1CFD9FF1E0EE126030EDB6A040EDB6A5D
:109BA000070EDB6A0C0EDB6A0D0EDB6A0E0EDB6A3B
:109BB0000F0EDB6A120EDB6A130EDB6AFB0EDBCFC5
:109BC000E6FFFC0EDBCFE6FF20EC3BF0E552E55272
:109BD000DF6A010EDB6A020EDB6A010EDBCF00F0EA
:109BE000020EDBCF01F0FF0E005C000E01583AE2DE
:109BF000070EDB0437E0010EDBCFE9FF020EDBCFFF
:109C0000EAFF000EE926050EEA22EFCF00F0DF5052
:109C1000E76EFD0EDBCFE9FFFE0EDBCFEAFFE7507C
:109C2000E926000EEA22EF50005C15E1010EDB2A66
:109C3000020E01E3DB2ADF2A0A0EDF5C0BE1010ED4
:109C4000F36E070EF3CFDBFF010EDB50E76E080E5D
:109C5000E7CFDBFFD0D7DF6A010EDB2A020E01E37C
:109C6000DB2ABBD7070EDB5001E058D1DF6A010EBB
:109C7000DB6A020EDB6A010EDBCF00F0020EDBCFE7
:109C800001F0FF0E005C000E01583AE2070EDB0403
:109C900037E0010EDBCFE9FF020EDBCFEAFF000E5B
:109CA000E926060EEA22EFCF00F0DF50E76EFD0E48
:109CB000DBCFE9FFFE0EDBCFEAFFE750E926000E1F
:109CC000EA22EF50005C15E1010EDB2A020E01E3EF
:109CD000DB2ADF2A0A0EDF5C0BE1010EF36E070EB2
:109CE000F3CFDBFF010EDB50E76E080EE7CFDBFFA3
:109CF000D0D7DF6A010EDB2A020E01E3DB2ABBD7D5
:109D0000070EDB5001E109D1080EDB50110FEA6AA2
:109D1000000FE96E060EEA22EF50E66ED950030FEF
:109D2000E96EDACFEAFFE552E750EE6EED6A030E18
:109D3000DBCF00F0040EDBCF01F000C001F0006AC1
:109D4000050E00C0DBFF060E01C0DBFF080EDB5076
:109D5000100FEA6A000FE96E060EEA22EF50E66E77
:109D6000D950030FE96EDACFEAFFE552E750EE6E05
:109D7000ED6A050EDBCF00F0060EDBCF01F0D95007
:109D8000030FE96EDACFEAFF0050EE260150ED2214
:109D9000080EDB50F50FE00BE83AE842E66ED950CA
:109DA0000A0FE96EDACFEAFFE552E750EE6EED6A90
:109DB0000A0EDBCF04F00B0EDBCF05F0050ED890BA
:109DC00004360536E806FBE11E0E0426000E0522C9
:109DD00004C0E6FF05C0E6FFCFEC3BF0E552E552DC
:109DE000F3CF00F0F4CF01F0026A036A0C0E00C05A
:109DF000DBFF0D0E01C0DBFF0E0E02C0DBFF0F0EFE
:109E000003C0DBFFD9500C0FE96EDACFEAFF040E76
:109E1000E76ED890000EEF36010EEB36020EEB36F1
:109E2000030EEB36E706F5E1D9500C0FE96EDACFF9
:109E3000EAFF040EE76ED890000EEF36010EEB3607
:109E4000020EEB36030EEB36E706F5E1D9500C0FA8
:109E5000E96EDACFEAFF040EE76ED890000EEF3617
:109E6000010EEB36020EEB36030EEB36E706F5E19C
:109E7000D9500C0FE96EDACFEAFF040EE76ED890E6
:109E8000000EEF36010EEB36020EEB36030EEB360C
:109E9000E706F5E10A0EDBCF00F00B0EDBCF01F099
:109EA000050ED89000360136E806FBE11C0E0026B0
:109EB000000E012200C0E6FF01C0E6FFCFEC3BF040
:109EC000E552E552100EF3CFDBFF110EF4CFDBFFAE
:109ED000100EDBCF04F0110EDBCF05F0066A076A27
:109EE000D9500C0FE96EDACFEAFFEE500424006E71
:109EF000EE500520016EEE500620026EEE50072057
:109F0000036E0C0E00C0DBFF0D0E01C0DBFF0E0E5A
:109F100002C0DBFF0F0E03C0DBFF09D1080EDB50D0
:109F2000110FEA6A000FE96E050EEA22EF50E66EA5
:109F3000D950030FE96EDACFEAFFE552E750EE6E33
:109F4000ED6A030EDBCF00F0040EDBCF01F000C0A2
:109F500001F0006A050E00C0DBFF060E01C0DBFF4A
:109F6000080EDB50100FEA6A000FE96E050EEA22B8
:109F7000EF50E66ED950030FE96EDACFEAFFE552F3
:109F8000E750EE6EED6A050EDBCF00F0060EDBCF7C
:109F900001F0D950030FE96EDACFEAFF0050EE2648
:109FA0000150ED22080EDB50F60FE00BE83AE842D4
:109FB000E66ED9500A0FE96EDACFEAFFE552E750B4
:109FC000EE6EED6A0A0EDBCF04F00B0EDBCF05F070
:109FD000050ED89004360536E806FBE11E0E042671
:109FE000000E052204C0E6FF05C0E6FFCFEC3BF003
:109FF000E552E552F3CF00F0F4CF01F0026A036AB4
:10A000000C0E00C0DBFF0D0E01C0DBFF0E0E02C008
:10A01000DBFF0F0E03C0DBFFD9500C0FE96EDACF68
:10A02000EAFF040EE76ED890000EEF36010EEB3615
:10A03000020EEB36030EEB36E706F5E1D9500C0FB6
:10A04000E96EDACFEAFF040EE76ED890000EEF3625
:10A05000010EEB36020EEB36030EEB36E706F5E1AA
:10A06000D9500C0FE96EDACFEAFF040EE76ED890F4
:10A07000000EEF36010EEB36020EEB36030EEB361A
:10A08000E706F5E1D9500C0FE96EDACFEAFF040ECE
:10A09000E76ED890000EEF36010EEB36020EEB366F
:10A0A000030EEB36E706F5E10A0EDBCF00F00B0EF0
:10A0B000DBCF01F0050ED89000360136E806FBE153
:10A0C0001C0E0026000E012200C0E6FF01C0E6FFC4
:10A0D000CFEC3BF0E552E552100EF3CFDBFF110E53
:10A0E000F4CFDBFF100EDBCF04F0110EDBCF05F059
:10A0F000066A076AD9500C0FE96EDACFEAFFEE5014
:10A100000424006EEE500520016EEE500620026E13
:10A11000EE500720036E0C0E00C0DBFF0D0E01C0D9
:10A12000DBFF0E0E02C0DBFF0F0E03C0DBFFD950BA
:10A13000030FE96EDACFEAFF000ED880EE54000E6E
:10A14000ED5401E301D1030EDBCF0FF0040EDBCFA2
:10A1500010F0140E0FC0DBFF150E10C0DBFF120E47
:10A16000DB6A130EDB6A030EDBCF0FF0040EDBCFCE
:10A1700010F01C0E0FC0DBFF1D0E10C0DBFFD9500E
:10A180001C0FE96EDACFEAFF000ED880EE54000E05
:10A19000ED5434E2140EDBCFE6FF150EDBCFE6FF05
:10A1A0004DEC37F0E552E5521C0EF3CFDBFF1D0EF0
:10A1B000F4CFDBFFD9501C0FE96EDACFEAFF000EB7
:10A1C000D880EE54000EED5418E21C0EDBCF0FF0D9
:10A1D0001D0EDBCF10F0120E0FC0DBFF130E10C0F0
:10A1E000DBFF1C0EDBCF0FF01D0EDBCF10F0140ECB
:10A1F0000FC0DBFF150E10C0DBFFC1D701014751B7
:10A20000046E056A140EDBCF02F0150EDBCF03F0EF
:10A21000020E025E000E035A02C00FF003C010F0DF
:10A2200004C014F005C015F0A6EC23F00D50010198
:10A230004325006E0E504421016E050E00C0DBFF69
:10A24000060E01C0DBFF160EDB6A170EDB6A180E66
:10A25000DB6A010EF36E1B0EF3CFDBFF1B0EDB5030
:10A26000000840E2050EDBCFE6FF060EDBCFE6FF7F
:10A2700020EC3BF0E552E552170EDB6A180EDB6A64
:10A280001B0EDB50000822E2170EDBCF00F0180E89
:10A29000DBCF01F0000E005C020E015817E2170E32
:10A2A000DBCFE6FF180EDBCFE6FF70EC3BF0E552AC
:10A2B000E552E76E1B0EE7CFDBFFDB50000805E23F
:10A2C000170EDB2A180E01E3DB2ADAD71B0EDB5050
:10A2D000000807E2050EDB2A060E01E3DB2A160E54
:10A2E000DB2ABCD70101010E0E6F0F6B106B0A0E3B
:10A2F000DBCF11F10B0EDBCF12F10C0EDBCF13F124
:10A300000D0EDBCF14F10E0EDBCF15F10F0EDBCFF0
:10A3100016F1120EDBCF17F1130EDBCF18F1140E6E
:10A32000DBCF19F1150EDBCF1AF1160EDBCF1BF1C7
:10A33000170EDBCF1CF1180EDBCF1DF1FB0EDBCFB0
:10A3400020F1FC0EDBCF21F1070EDB50006E016A1D
:10A3500000C0F3FF01C0F4FF00D0D9CFE1FFE55208
:10A36000E7CFD9FF1200D9CFE6FFE1CFD9FF180E12
:10A37000E126DF6A010EDB6A020EDB6A030EDB6A8E
:10A38000040EDB6A010EF36E130EF3CFDBFF140E27
:10A39000DB6A150EDB6AD950010FE96EDACFEAFFEE
:10A3A000EE50ED1020E1200EDF5C1DE2DF500101D8
:10A3B000016A4125006E4251012200C0E6FF01C042
:10A3C000E6FFF30EE66E040EE66EA6EC48F0E1063C
:10A3D000E106E106E106DE52F3CFDEFFF4CFDDFF5A
:10A3E000DD52DF2AD8D7DF6A080EDF5C19E2DF50C2
:10A3F000EA6A010FE96E010EEA22EF50E66ED950CB
:10A40000050F006EDACF01F0DF500F01EA6B002478
:10A41000E96F0150EA23E552E750EF6EDF2AE4D7F7
:10A42000090EDF6E0C0EDF5C19E2DF50EA6A010FE5
:10A43000E96E010EEA22EF50E66ED950050F006E6C
:10A44000DACF01F0DF040F01EA6B0024E96F01505D
:10A45000EA23E552E750EF6EDF2AE4D7010EDBCFA7
:10A46000E6FF020EDBCFE6FFD950050FE66EDACF2E
:10A47000E6FFA6EC48F0E106E106E106E106030E80
:10A48000F3CFDBFF040EF4CFDBFF01014751046E75
:10A49000056A010EDBCF0FF0020EDBCF10F0435147
:10A4A0000F5C026E44511058036E02C00FF003C0DF
:10A4B00010F004C014F005C015F00AEC22F00FC033
:10A4C00000F010C001F0020E0026000E0122110E55
:10A4D00000C0DBFF120E01C0DBFFD950130FE96E85
:10A4E000DACFEAFF000ED880EE54000EED5401E3FF
:10A4F00088D0D950030FE96EDACFEAFFEE50ED10A5
:10A5000001E07FD0110EDBCFE6FF120EDBCFE6FFBE
:10A510004DEC37F0E552E552130EF3CFDBFF140E8E
:10A52000F4CFDBFFD950130FE96EDACFEAFF000E4C
:10A53000D880EE54000EED5463E201014751046EE1
:10A54000056A130EDBCF02F0140EDBCF03F0020E10
:10A55000025E000E035A02C00FF003C010F004C0E8
:10A5600014F005C015F0A6EC23F00D5001014325B1
:10A57000006E0E504421016E010E00C0DBFF020E82
:10A5800001C0DBFF150EDB6A01014751F36E150EAA
:10A59000DBCFF4FFF350F45C27E2D950030FE96EF0
:10A5A000DACFEAFFEE50ED101FE1010EDBCFE6FF40
:10A5B000020EDBCFE6FFD950050FE66EDACFE6FFDD
:10A5C000A6EC48F0E106E106E106E106030EF3CF52
:10A5D000DBFF040EF4CFDBFF010EDB2A020E01E3EA
:10A5E000DB2A150EDB2AD0D7130EDBCF0FF0140EAB
:10A5F000DBCF10F0110E0FC0DBFF120E10C0DBFF1F
:10A600006CD7030EDBCF00F0040EDBCF01F00101AD
:10A610000050435D0150445923E2010EDBCFE6FFB9
:10A62000020EDBCFE6FFD950050FE66EDACFE6FF6C
:10A63000C6EC4DF0E106E106E106E106160EF3CFA9
:10A64000DBFF170EF4CFDBFFD950160FE96EDACF20
:10A65000EAFFEE50ED1002E0FF0E04D0000E02D033
:10A66000000E00D0D9CFE1FFE552E7CFD9FF1200AD
:00000001FF
